S02B0000433A2F4D4A42432F496E7465726E616C2F755461736B6572426574612F4170706C69636174696F6E73
S10B200000000120E97C00004E
S1132008034B1868042814BF0020012070470000FF
S113201850050020024B1A78024B1A7070470000D2
S11320281C0500201D05002070470000024A1368A3
S113203883F0020313607047FCD3054010B50023F6
S113204884B08DF808301E4BC1B21A68002092F88B
S113205821301C4C8DF80B304FF04003ADF80430A0
S11320684FF48073ADF8063061238DF80C3092F884
S11320784B308DF80E3092F84C308DF80F30938B2E
S11320886A46009301238DF80D3002F0D1FD2070CB
S113209890B10521002202F077F9009B13F0400F5C
S11320A80AD040F204410022207802F06DF9207829
S11320B88121002202F068F9024B187804B010BD9F
S11320C84C050020A00B002000B50949094B0A78EB
S11320D81A7028B1022818BF4FF0FF3306D102E066
S11320E8054B1B7802E001F00DFE00E00B7000BD0B
S11320F81D0500201C050020A00B002000B5024887
S113210803F062FB00BD00005C8F0000044B012259
S113211800B51A60612004F0CDFBFFF7EFFF00BDA6
S11321285005002000B50249182202F067FA00BDE4
S11321387C8F0000182210B548F20400134903F0FC
S1132148F3FC0028A8BF4FF4004013DA0420182237
S11321580E4903F0E9FC002801DB00200AE00B48E3
S1132168FFF7E0FF0A4B0B4918683C2202F046FAD5
S1132178002408E0064B044640F01C0080B21968AD
S11321883C2203F0D1FC204610BD0000A10B002026
S113219848050020208F000030B5012886B0224C65
S11321A820D118222149684602F028FAFFF7C2FF15
S11321B8182205461D49206802F020FA1C4B1B68AA
S11321C81B7A13F0020F15D004A90422194802F04F
S11321D815FA03A90422184802F010FA174802A9AC
S11321E8042205E0FFF7A6FF1049054620681822D7
S11321F802F004FA0C4C18222168114802F0FEF986
S11322080B4B2068196818303C2202F0F7F9206853
S1132218037E082B04D018300A493C2202F0EEF958
S1132228284606B030BD00004C050020A10B002054
S113223848050020B10B0020AD0B0020A90B00209D
S1132248B90B0020208F0000182200B548F20400C2
S11322580C4903F069FC002809DA0420182209490A
S113226803F062FC002802DA0648FFF75BFF054B1F
S11322781A78597842EA012242F004021A70120AC2
S11322885A7000BDA10B002080B2134B202800B562
S113229818800BD002D8D8B1082805E0802817D0B8
S11322A8B0F5807F09D0402815D111E0612041F2B2
S11322B87071062204F024FB0DE0062261204FF41D
S11322C8966104F01DFB054B1A78054B1A7002E061
S11322D8612004F0EFFA00BD80050020A00B002067
S11322E81D05002000B5044B0021187802F0B0F851
S11322F8024B01221A6000BDA00B002050050020EB
S113230800B5002387B000930F230293F0230393AF
S113231803F1005303F5FE431033049306238DF8A9
S11323281630084B0222069368464FF002038DF8D4
S113233804208DF80520ADF8143005F041F907B0F4
S113234800BD00006005002070B5754C90B023688E
S1132358867B002B40F09D803C2003F07BFC714B76
S11323681860542003F076FC6F4B18600020FFF7C8
S113237813FFB0F5004F08D161204FF41661032212
S113238804F0BEFA0423236003E001232360FFF76B
S1132398B5FE00F057FA6D20042104F0EBFA03208F
S11323A8FFF74CFE002800F0B980604B60481A78AB
S11323B8604B1A7002F01AFB7520042104F0DAFA53
S11323C8FFF79EFF5C4801230371022383724FF0D9
S11323D80B03C3800023036003896433038105F07E
S11323E8EFF856E09DF8032012B1012A4BD11AE008
S11323F89DF80430032B03D1032003F051FB0AE0BA
S1132408062B06D1494B4D491878162202F044FA96
S11324183FE0832B02D105F0E1FB3AE06C2B38D185
S1132428FFF76EFF35E09DF80430DF2B05D13C49FA
S11324380B68082B08BF0A602BE05E2B29D14048A3
S113244802F0D4FA3F4802F0D1FA3F4D00243F4845
S113245802F0CCFA00210022204602F0DDFA3C48C2
S113246802F0C4FA0134822135F8020B02F0C6FAEC
S1132478102CECD1374802F0B9FA612064216C229F
S113248804F03EFA05E09DF804203046694601F060
S113249897FF3046694605226C4601F091FF0028F3
S11324A8A0D11F4B1B6813F0370F37D01F4B187878
S11324B801F09EFF40BB31E0274B1B8813F4804F8B
S11324C804D06846214601F04DFC1DE068462146CB
S11324D800F046FE214B1B888BB968462146002232
S11324E801F012FB80B14FF4807000F0C7FE02289F
S11324F80AD130781A49172202F0CEF904E0684666
S11325082146002201F000FB084E6946307840223B
S113251801F056FF6D4604460028CDD110B070BDB9
S113252850050020480500204C050020A00B002081
S1132538C88E00001D05002054050020AC8F000043
S1132548EC8E0000FC8E000060050020088F00005F
S113255800980000389800008205002080050020BB
S1132568948F0000013103E001319A420FD1013008
S113257811F8013C0278002BF6D1202A07D8013043
S113258810F8013C0130202BFAD0023800E000207A
S11325987047000000B503685A1C02E00368013361
S11325A8036012F8013C0132202BF7D0511E4FF082
S11325B8000C4FF0030E15E0303BDAB2092A01D9BA
S11325C8D31FDAB24FEA0C139BB202F00F0243EAAC
S11325D8020C03680EF1FF3E01330131BEF1FF3FE7
S11325E8036003D011F8013C2F2BE5D8604600BDE9
S11325F8013010F8012C01300F2A14BF00230123E5
S1132608202A08BF43F00103002BF2D10238704797
S113261870470000064BC0B231381A68C0B20123B3
S11326288340DBB21A420CBF00200120704700002F
S1132638FCD30540064BC0B231381A68C0B2012336
S11326488340DBB21A4214BF002001207047000007
S113265800D40540C0B2C9B2303864295FFA80FC9E
S11326680AD002D8612904D124E0692904D06F2949
S11326780DD04FF0FF301EE0BCF1030F1AD8012231
S113268802FA0CF20C48036823EA020308E0BCF1DE
S1132698030F0FD8012202FA0CF207480368134308
S11326A8064903600B6813430B60054B02681B68FB
S11326B883F84D200020704700D405401CD5054000
S11326C84C050020C0B261380F2809D8DFE800F0B3
S11326D80A0C0E10121416181A1D2125292D31352D
S11326E800202FE0184B0EE0174B0FE0164B11E0BB
S11326F8154B13E0144B15E0134B17E0124B19E07C
S1132708114B1BE0114B1B681AE0104B1B685B084C
S113271816E00E4B1B689B0812E00C4B1B68DB0889
S11327280EE00A4B1B681B090AE0084B1B685B098F
S113273806E0064B1B689B0902E0044B1B68DB0997
S113274803F0010070470000FC930540FCA305401A
S1132758C0B2A0F161030F2B41D8DFE803F0080AE7
S11327680C0E10121416181D22272C31363B224A3F
S11327780EE0214A11E0204A14E01F4A17E01E4ADD
S11327881AE01D4A1DE01C4A20E01B4A23E01B4AAC
S1132798136883F0010321E0184A136883F00203E5
S11327A81CE0164A136883F0040317E0134A1368FD
S11327B883F0080312E0114A136883F010030DE054
S11327C80E4A136883F0200308E00C4A136883F068
S11327D8400303E0094A136883F080031360084B3D
S11327E8A0F16102196801239340B1F85020002038
S11327F85340A1F850307047FC930540FCA30540B2
S11328084C050020C0B251B10A4A136843F02003B2
S11328181360C03A136823F02003136002E0064BE8
S11328281B681840054B18601A68054B1B6883F829
S11328384E20704708E10F4000D40540FCD3054002
S11328484C05002070B5C14901250A68302492F866
S11328584E3092F84D6006EA030382F84E300B6856
S1132868012193F84E00FFF7CDFF2E4214BF6F21CC
S1132878692120460134FFF7EDFE382C02D06B00A5
S1132888DDB2F2E7B24A0121136843F0060313608C
S1132898AE4B1B68B3F8500008425FD0802931D092
S11328A810D808292ED005D802292BD0042929D0DC
S11328B8012904E0202925D0402923D0102940F0FB
S11328C8BD801FE0B1F5006F2FD00AD8B1F5007FA5
S11328D821D0B1F5806F23D0B1F5807F40F0AE8070
S11328E814E0B1F5005F2AD004D8B1F5805F40F058
S11328F8A5801FE0B1F5804F26D0B1F5004F40F018
S11329089D8026E0934A13680B438DE0924A13682E
S113291843F0010388E0904A136843F0020383E01C
S11329288D4A136843F004037EE08B4A136843F02E
S1132938080379E0884A136843F0100374E0864A70
S1132948136843F020036FE0834A136843F040039D
S11329586AE0814A136843F080036DE080293CD023
S113296810D8082931D006D802292AD004292AD017
S1132978012963D123E020292BD040292BD0102909
S11329885CD124E0B1F5006F3BD009D8B1F5007FE4
S11329982DD0B1F5806F2FD0B1F5807F4ED121E0D5
S11329A8B1F5005F37D003D8B1F5805F46D12DE08B
S11329B8B1F5804F34D0B1F5004F3FD138E0654AC6
S11329C811E0644A14E0634A17E0624A1AE0614A73
S11329D81DE0604A20E05F4A23E05E4A136823F062
S11329E8800321E05C4A136823F001031CE05A4A7F
S11329F8136823F0020317E0574A136823F004030B
S1132A0812E0554A136823F008030DE0524A13688C
S1132A1823F0100308E0504A136823F0200303E06E
S1132A284D4A136823F0400313604B0099B233E70F
S1132A38494A136823F08003136004E04B0099B2F9
S1132A4800297FF429AF414B62211B68A3F8500089
S1132A5810E04B1CD9B24B1EDBB2613B0F2B71D873
S1132A68DFE803F0080A0C0E1012141618232E3986
S1132A78444F5A65394A0EE0384A17E0374A20E08D
S1132A88364A29E0354A32E0344A3BE0334A44E0E6
S1132A98324A4DE0324A136843F001031360A2F549
S1132AA88E72136843F001034BE02D4A136843F018
S1132AB802031360A2F58E72136843F0020340E028
S1132AC8274A136843F004031360A2F58E7213684F
S1132AD843F0040335E0224A136843F00803136003
S1132AE8A2F58E72136843F008032AE01C4A13689F
S1132AF843F010031360A2F58E72136843F01003B9
S1132B081FE0174A136843F020031360A2F58E727E
S1132B18136843F0200314E0114A136843F0400398
S1132B281360A2F58E72136843F0400309E00C4A5F
S1132B38136843F080031360A2F58E72136843F0A0
S1132B4880031360702984D970BD00004C050020EF
S1132B5808E10F40FC930540FCA305401C95054083
S1132B681CA505408288130A43EA0223838003686C
S1132B781A0A02F47F4242EA136242EA03621B021F
S1132B8803F47F0313430360704700007047000099
S1132B980020704730B50246481C10F8013C01304B
S1132BA82B2BFAD00238042A16D0072A27D0032A56
S1132BB82AD1164C256801F009FD85F84B002468D4
S1132BC894F84B30632B01D9632302E0092B1BD8FB
S1132BD80A2384F84B3017E00C4C256801F0F6FC06
S1132BE885F84C00246894F84C30632B01D963238E
S1132BF802E0092B08D80A2384F84C3004E0034B7C
S1132C081C6801F0E3FCE08330BD00004C050020A3
S1132C1810B50F4B024619688B78CC78C87904EB49
S1132C2803248B7991F804C000EB03204B7902212B
S1132C381B0403EB0C63C01801F0EEFEA4B20246B9
S1132C482D2302F8013B2046022101F0E5FE10BDC8
S1132C584C0500202A4B70B519682AA318CBA1FB90
S1132C6803562AA318CB35090246A5FB03010C0C0D
S1132C782046002101F0D0FE04EB44044FF0200C60
S1132C880246442302F801CBC4EB041443706123C5
S1132C985370511C7923C4EB04144B70481C7323E0
S1132CA8A5EBC415421C43701AA318CBA5FB03015A
S1132CB8CC0A82F801C000210232204601F0ACFEA1
S1132CC8C4EB0414C4EB0414A5EB0415024613A3C3
S1132CD818CBA5FB03013A264C0902F8016B022123
S1132CE8204601F099FEC4EB04140246A5EB8405C2
S1132CF802F8016B2846022101F08EFE70BD000027
S1132D08DC0B0020CDCCCCCCFFFFFFFF07452EC247
S1132D18FFFFFFFFC5B3A291FFFFFFFF89888888E3
S1132D28FFFFFFFF10B5CCB201F060FE094801F0C7
S1132D385DFE094B1B6893F820301C4204D00748F9
S1132D4801F054FE012003E0054801F04FFE002085
S1132D5810BD0000449400004C0500204894000075
S1132D6854940000F0B5684B81B01B6805468EB2D8
S1132D78032B00F2A280DFE803F002494782634C88
S1132D8823683BB94FF40070042102F037FF604B0D
S1132D98206018605F4B00221A605F4B1A6022683B
S1132DA85B4B1A60584B01221A602FE0002E73D037
S1132DB815F8013B013201F8013B731E082A9EB243
S1132DC828D1534B1960534B1A60504B1C6820464A
S1132DD8FFF7C8FEA28841F234239A4261D12268DF
S1132DE8494FB2F5803F62D24C4B08321A604C48C6
S1132DF802F038FE4B4B186002233B604A4801F04E
S1132E08F5FD2046FFF7AEFE6F1C32E0404B196813
S1132E18404B1A68B2F5007FC8D33D4B19603D4B4F
S1132E281A60F1E7002E48D0394A4D1C136817F888
S1132E38012CB5F5007F03F8012B354A1360354B97
S1132E481D6013D1394801F0D1FD304C354B2A4669
S1132E581868216802F08AFD2F4A13685B19136009
S1132E682C4A002313602368294A1360731E9EB2F8
S1132E780137284B1968B1F5007FD3D31DE0D6F18B
S1132E88010338BF0023002814BF002303F0010303
S1132E98002B37D0002208E01D4B19601D4B1A6027
S1132EA830E0234801F0A2FD0322174BF7E721483D
S1132EB801F09CFD03233B6024E0174BD3F800C0CA
S1132EC8164B1A68134B1B68634493421AD30523A1
S1132ED862458DF8033007D9124BCCEB020218680F
S1132EE80A4B196802F042FD0E4B0DF103011868F4
S1132EF802F088FC104801F079FD61202821832222
S1132F0803F0FEFC01B0F0BD9C0500208C050020F8
S1132F1888050020980500209005002094050020CD
S1132F2898940000840500209C940000AC94000050
S1132F38609400007C940000B094000010B5084C24
S1132F482068FFF7EFF8206806220230054901F0EF
S1132F5855FB2068044918303C2201F04FFB10BD92
S1132F684C050020A30B0020208F000010B5C0B230
S1132F78022884B002D0042825D11EE0134801F0A9
S1132F8835FD6846FFF744FE684601F02FFD1048FA
S1132F9801F02CFD0F4801F029FD0F4801F026FD32
S1132FA80B4801F023FD0D4801F020FD0C4B6C4645
S1132FB81868363001F01AFD05E0094B1422186828
S1132FC8363001F01BFB04B010BD0000CC940000A7
S1132FD860950000E0940000BC8E0000F4940000AA
S1132FE84C050020022830B50546214C11D1214B4F
S1132FF820681B6890F820201B7A02F0020203F074
S113300802039A4221D11C49182201F003FBE0B9BA
S11330181DE01822216848F2040002F063FD2168CB
S11330283C22183148F21C0002F05CFD012D0AD044
S1133038022002F035FD0F4B3C2218680C4B19682E
S1133048183101F0DBFA002010E001200EE0084CF2
S11330581822216848F2040002F044FD21683C2249
S1133068183148F21C0002F03DFDE1E730BD0000D4
S11330784C05002048050020B90B0020204B10B552
S11330881868204B828B19688B889A4212D190F861
S11330984B2091F833309A420CD190F84C2091F897
S11330A834309A4206D190F821204B7AD41A18BFAA
S11330B8012400E0012490F82000097A00F0280295
S11330C801F028039A4200F0040201F0040318BF37
S11330D844F002049A4200F0100201F0100318BFF1
S11330E844F004049A4218BF44F008040120FFF78E
S11330F853F814F0010F02D00420FEF79FFF10BD0F
S11331084C05002048050020F0B5144B81B01B681D
S1133118002693F84D70B3F85030012500933124FC
S11331282046FFF777FA00B12E430134392C02D038
S11331386B00DDB2F4E7FFF7A1FF084A002013682B
S113314883F84D70136883F84E601368009AA3F8E7
S11331585020FFF747FF01B0F0BD00004C050020E8
S113316800B5044B84468AB21878614601F094FB92
S113317800BD0000A00B0020F0B5374A374D137886
S113318888B003EB43039B0003EB05025C591379F6
S1133198074656790DF1050020211B22009301F002
S11331A825FA4FB1002201E00C340132C2EB0603C8
S11331B8BB42F9DC1E4645E0294801F017FC264AC3
S11331C8137803EB430305EB8303986801F00EFCC3
S11331D8244835E041F26D022878402101F0D4F802
S11331E8214B721C01201A6033E0204B1B88202BD2
S11331F804D01F4B1B88B3F5805F07D11D4D0021F8
S11332082878422201F048FB0028E3D054F80C0C3B
S113321801F0ECFB009D0346A8420DF10501154A97
S113322802DB1078012204E0009D1078C3EB05024C
S113323892B201F031FB54F8080C01F0D7FB0E48A8
S113324801F0D4FB0C34013ECFD2074B00221A60A4
S1133258002008B0F0BD0000A205002078A00000FE
S11332680C95000010950000A4050020800500209E
S1133278820500201D0500206095000080B2B0F58D
S1133288807F00B510D0B0F5006F1C4B1CBF4FF405
S113329800721A8010D11B88002B2DD1184B1B8863
S11332A853BB184B188015E0164B1B8823BB134BD4
S11332B81B880BBBFEF7E8FF114B1B88B3F5807F17
S11332C803D12020FEF7E0FF0AE00E4B1B88B3F57C
S11332D8006F05D10B4B4FF480521A8000F012FD99
S11332E802200021FFF742FE074B00221A7000203B
S11332F8FFF742FF002000E0022000BDA0050020E7
S11333088005002082050020A205002030B504466F
S1133318CDB21048214601F091F948B10E48214632
S113332801F08CF958B10D4801F060FB01200FE061
S11333380B4B1A6892F8203045EA030305E0084B62
S11333481A6892F8203023EA050382F82030002016
S113335830BD000028950000309500003895000025
S11333684C050020F0B5C0B287B01546C9B208288C
S113337800F24483DFE810F009002D001A013D0132
S11333884203AB01EC02F102F60029B1042907D18A
S11333980122DFF870361A700020FFF7EDFE2EE3E5
S11333A8052901D10222F4E7062901D10322F0E715
S11333B8072901D10422ECE7092901D10522E8E70C
S11333C80A2901D10622E4E70D2940F017830022D7
S11333D8DFE70C2900F21283DFE811F00D0010007A
S11333E89D001003870055001003100310031003F9
S11333F832003E00840004F0F1FBFFE2DFF8080627
S113340801F0F4FADFF8040601F0F0FADFF8000638
S113341801F0ECFA02F0E2FB822101F0EFFADFF8A6
S1133428F40501F0E3FA02F0CDFB822101F0E6FA9B
S1133438DFF8E40501F0DAFA02F0B6FB82211DE1B7
S11334486846FFF707FC00230370DFF8D00501F096
S1133458CDFA6C466846CFE22B78313BDBB2032BBE
S113346888BFDFF8BC0500F2C782DFF8B80501F0B1
S1133478BDFA2878FFF7DEF810B9DFF8AC05BBE22F
S1133488DFF8A805B8E22878A0F13103DBB2032BF2
S113349830D8FFF7CFF810B1DFF89405ACE2002775
S11334A8012631242046FFF7B5F800B1374301342B
S11334B8352C02D07300DEB2F4E7284601F06CF82C
S11334C8C0B2013801238340681CDCB201F064F8FF
S11334D801280CBF47EA040027EA04000021FFF78B
S11334E891F98BE2FFF710FE88E22B78313BDBB2CF
S11334F8032B02D9DFF83C057EE2DFF83C0501F036
S113350875FA2878FFF786F810B1DFF8300573E20A
S1133518DFF82C0570E2284601F03EF82B780246C5
S1133528202B18BF284605D12846013009E0202B56
S1133538FBD001300378002BF9D1F6E701302029BC
S113354804D110F8011C0029F8D108E039B102F1BE
S11335582F00C0B2FFF77EF8002800F04F82DFF892
S1133568E40449E2C8B218B1012840F047820AE0ED
S1133578DFF8D40401F03AFADFF8D024138843F4CE
S1133588804313803AE2DFF8C4442388B3F5805FAC
S113359818BFDFF8BC0440F02F82DFF8B80401F04C
S11335A825FA238843F40053238027E2C8B250B194
S11335B8032840F02382DFF8A03428461C6801F071
S11335C805F8E0831AE2DFF894442388042B07D132
S11335D8DFF88C0401F00AFA4FF0100222800DE2A1
S11335E8DFF868344FF000021A800020FEF74CFE22
S11335F804E20595072900F20182DFE801F0042BB3
S11336085259165E634305AC2046FEF7C3FF0546D0
S11336182046FEF7BFFF07A901F8010D012228463D
S113362802F060FADFF83C04E6E105AD2846FEF74F
S1133638B1FF04462846FEF7ADFF44F4004407A949
S1133648A4B201F8010D0122204602F04BFADFF87A
S11336581804D1E105A8FEF79DFF01220DF11B0115
S113366802F062FA0028B8BFDFF80004C0F2C4818F
S1133678FF4801F0BBF99DF81B00012101F0BEF9D8
S1133688FC48B9E1F44CFC491822206800F0B6FF64
S11336982068FA4B183019683C2200F0AFFFF8484C
S11336A8AAE1FFF74BFC0020FFF79CFCF548A3E1D7
S11336B8012002F0F5F9F4489EE1022002F0F0F945
S11336C8F24899E10020FFF78DFCF14894E1CCB26F
S11336D8162C00F29381DFE814F017005E0028002E
S11336E83D007F00910191019101910191019101A6
S11336F8910191019101910191019101A000910120
S1133708910191011E011E01D34BE24E1F68002452
S11337183046294600F092FF002800F00F8101345A
S113372807360C2C00F05981F2E72878372805D1A0
S1133738C94B1A68938B43F0010309E0382818BF72
S1133748D54840F05981C44B1A68938B23F0010380
S11337589383F9E0C04BD14E1C68002730462946B4
S113376800F06CFF88B9A38B4FF6F97203EA0202E2
S1133778A2831FB1012F40F0E78002E042F0040366
S113378801E042F00203A383DEE001370536032F8C
S113379800F02581E2E7B04BC14E1C680027304693
S11337A8294600F04BFF88B9A38B4FF6E77203EA6A
S11337B80202012FA28303D0022F40F0C58002E049
S11337C842F00803DFE742F01003DCE70137043670
S11337D8032F00F00681E2E79F4BB24E1C680027D6
S11337E83046294600F02AFF88B9A38B4FF69F720A
S11337F803EA0202012FA28303D0022F40F0A4801F
S113380802E042F04003BEE742F02003BBE7013781
S11338180836032F00F0E780E2E7A34801F0E6F852
S1133828A24801F0E3F88C4B1B6893F821300B2B6A
S113383897BFC3EBC3009E48964BC01801F0D6F857
S11338489C4801F0D3F8844B1B689B8B13F0010F41
S113385814BF9948994801F0C9F8994801F0C6F885
S11338687D4B1B689B8B13F0020F01D0012304E0EE
S113387813F0040F0CBF0223002303EB8300874BD0
S1133888C01801F0B3F88F4801F0B0F8724B1B6808
S11338989B8B13F0100F01D0022302E0DB0803F026
S11338A801037F4800EB830001F0A0F8864801F08B
S11338B89DF8694B1B689B8B13F0400F01D00124C2
S11338C804E013F0200F00F0908002247F4801F0F8
S11338D88DF8744800EBC40001F088F85E4C754814
S11338E801F084F87A4801F081F82368002193F8FC
S11338F84B00002201F090F8764801F077F87648FA
S113390801F074F82368002193F84C00002201F0B8
S113391883F8704870E0284600F058FEC0B2632867
S113392801D9632002E0002808BF01204A4B152C66
S113393804BF1B6883F84B0006D002E087F82140D7
S113394802E01B6883F84C000420FEF777FB55E07F
S113395808462946FFF70AFB50E006294ED8DFE857
S113396801F004070A1018130D00284610210DE071
S1133978284602210AE02846042107E02846402177
S113398804E02846082101E028462021FFF7BEFC70
S113399834E0524801F02AF840215148FFF7C2F9AF
S11339A804215048FFF7BEF94F480821FFF7BAF938
S11339B818B14E482021FFF7B5F94D481021FFF7FB
S11339C8B1F9D8B14B4801F011F8234B00211B6819
S11339D80022D88B01F020F80DE047480CE0474856
S11339E80AE0474808E0474806E0384800F0FEFF88
S11339F82C4800F0FBFF2F4800F0F8FF002007B028
S1133A08F0BD0000A20500204C950000649500005C
S1133A187C9500008C95000094950000A895000002
S1133A28D0950000E4950000F89500000496000085
S1133A381C9600000C9600002C9600003C96000092
S1133A4840960000449600004C9600008205002031
S1133A5884960000A49600004C050020A0050020D0
S1133A68BC960000C8960000DC9600000C97000085
S1133A78F496000060950000A10B00204805002082
S1133A883097000054970000749700009097000046
S1133A98B0970000D8A00000C89700002CA100002F
S1133AA83BA1000047A10000E0970000FC9700003C
S1133AB8049800003898000010980000149800003A
S1133AC818980000209800002C9800003C980000EA
S1133AD84C980000589800005C9800006898000012
S1133AE88098000094980000A0980000AC9800000A
S1133AF8C8980000D8980000F498000010990000B5
S1133B08249900003C990000F0B589B283B00025DF
S1133B180290009201918BE0029B1A78082A0AD13C
S1133B284A4A1378002B00F08380013B13704848FD
S1133B3800F05CFF7CE0D2F1010338BF00230A2ABD
S1133B4814BF1F4643F00107002F71D13F4C414E6B
S1133B5821787254029A13780D2B5FD10A230098A6
S1133B687354FEF7B1FA23783B490133D8B23B4B7F
S1133B781B7803EB43039B0003EB01025D58731EA0
S1133B88C754009B52793BB9354B1B88002B3BD05B
S1133B9813F4806F38D106E0009B022B03D1314B1C
S1133BA81B88002B30D000282BD0144611E029683C
S1133BB82848FEF7D7FC024650B1287A697AFFF7FD
S1133BC8D1FB10B9284800F011FF009AE2B913E0BC
S1133BD80C35013CEBD2254C1E482168FEF7C2FC8B
S1133BE8024670B1207A617AFFF7BCFB10B91E480F
S1133BF800F0FCFE009B3BB9194B1888FEF744FB08
S1133C0802E01B4800F0F2FEFEF704FA0F4B002214
S1133C181A70029A01250132029209E04B1C029A99
S1133C28DBB20132272B2370029201D92723237098
S1133C38019A531E9BB20193019A4FF6FF739A425D
S1133C487FF46AAF284603B0F0BD0000A805002041
S1133C5875A00000A905002078A00000A205002096
S1133C68800500208205002048960000CCA00000B2
S1133C784496000030B5857B88B031E09DF8033068
S1133C88012B02D0412B25D112E09DF80430DF2B03
S1133C9826D1184B186810B1FFF76EFA20E0164ABF
S1133CA8137813F0010F1CBF23F00103137017E0FE
S1133CB89DF804202846694600F082FB9DF80030F0
S1133CC8042B08BF0D4802D0032B09D10C4800F07F
S1133CD88DFE05E09DF804202846694600F070FB37
S1133CE82846694605226C4600F06AFB0028C5D1BF
S1133CF808B030BDA4050020D10500205899000063
S1133D086C990000024B1A78024B1A707047000035
S1133D18D90500201D0500204FF012030380014837
S1133D287047000013A500004FF0430303800148C7
S1133D3870470000D0A4000080B205280CD8074BB7
S1133D4853F82020137823B9032805D1044B1A68A3
S1133D58137810460B8000E000207047B8A40000D8
S1133D68DC05002000B5044B84468AB21878614605
S1133D7800F092FD00BD0000D9050020F0B506460C
S1133D888FB22AB1022A01D1002073E0002040E05A
S1133D98017821F08003212B64D1C279837911F051
S1133DA8800F43EA0223344A1380427807D0212A39
S1133DB858D17520012100F0D9FE002023E0202AE3
S1133DC802D0222A4ED103E02C4B06201A701AE0A6
S1133DD8837813F0020F2A4B02D01878812101E06E
S1133DE818788221002200F0CFFAB37813F0010F7B
S1133DF8234B02D01878842101E018788821002206
S1133E0800F0C2FA0320082F34D9A7F108039FB29F
S1133E180836194B1A88EAB1184B1B78202B15D190
S1133E28072A34BF14460724BDB2164BA542C4EB77
S1133E38030019D8073031462A4600F0DFFBA542B3
S1133E4803D37520022100F091FE03200A4A138847
S1133E589F4204D3084B4FF000021A800AE0DB1B90
S1133E68138007E0042005E007303146224600F0BD
S1133E78C5FBE6E7F0BD0000D6050020D505002007
S1133E88A00B0020E0050020F0B5DFF8AC34807BFF
S1133E981B78A6B00090002B40F0ED81DFF89C342D
S1133EA8DFF89C541E6806F11E0000F0F1FB2B6835
S1133EB84BB944000234E4B2204601F0CBFE03239C
S1133EC82860047043702B6806F11F009A1C04E0F4
S1133ED8002302F8027C02F8013C10F8017C02324B
S1133EE80130002FF4D1DFF85C3421AC4FF001022B
S1133EF84FF00005ADF88E20219303267523002189
S1133F08224605208DF896308DF89270ADF88A50C7
S1133F18ADF888508DF894508DF8956000F088FEBF
S1133F28DFF814344FF48072187002238DF892303D
S1133F384FF001038DF89330ADF888204FF040031B
S1133F484FF40072ADF89030ADF88C204FF48063D4
S1133F58002122460520ADF88A30219700F068FE3A
S1133F68F94B4FF000021870ADF88A204FF0400367
S1133F78052000212246ADF890308DF892608DF826
S1133F8893508DF89650219700F052FEEF4B18701D
S1133F9871E19DF80730012B03D0752B40F06B813C
S1133FA852E19DF80830CD2B2DD005D8012B30D007
S1133FB8022B40F0608199E0CE2B11D0CF2B40F03A
S1133FC85A81E34C23884BB1E24B00201A78E24B28
S1133FD81A70FEF759F94FF000032380DF4848E1CF
S1133FE8DB4C23884BB1DB4B00201A78DA4B1A7070
S1133FF8FEF74AF94FF0000222800120002101F067
S1134008AFFFD74835E10220002101F0A9FFD548C8
S11340182FE1D54B1B6893F821300C2B22D8DFE80D
S113402803F00C0F1215181B1E2124272A070A0057
S11340384FF4613221E0CD4A1FE04FF496721CE040
S11340484FF4167219E04FF4966216E04FF41662B4
S113405813E04FF4965210E04FF416520DE04FF46B
S113406861520AE04FF4964207E04FF4164204E026
S11340784FF4614201E04FF4E132BD49130A4B7039
S1134088130C8B70130ECB70B74B0A701B689B8B89
S113409813F0010F01D0072300E008238B71B24B02
S11340A81B689B8B13F0020F03D0B14B02225A7189
S11340B805E013F00403AE4A18BF01235371AA4B59
S11340C81B689B8B13F0080F03D0A94B01221A71AC
S11340D805E013F01003A64A18BF02231371964B88
S11340E8A3491878072200F0D7FBC4E0A04B5A78FC
S11340F8197841EA0221DA789B781B0443EA0263BF
S11341081943B1F5613F03D9974B1A680C234EE064
S1134118B1F5E13F03D9944B1A680B2347E0B1F595
S1134128614F03D9904B1A680A2340E0B1F5164F42
S113413803D98D4B1A68092339E0B1F5964F03D991
S1134148894B1A68082332E0B1F5615F03D9864BBD
S11341581A6807232BE0B1F5165F03D9824B1A6856
S1134168062324E0B1F5965F03D97F4B1A6805232B
S11341781DE0B1F5166F03D97B4B1A68042316E0CA
S1134188B1F5966F03D9784B1A6803230FE0B1F59C
S1134198167F03D9744B1A68022308E0B1F5967F99
S11341A8714A02D91268012301E01268002382F8D7
S11341B821306F4B6C4A9B79072B0BBF126812682E
S11341C8938B938B0CBF43F0010323F00103938378
S11341D8674B5B79012B09D0022B634A0ED1126815
S11341E8938B43F0020323F004030BE05E4B1A683D
S11341F8938B23F0020343F0040303E01268938BC8
S113420823F0060393835A4B1B79012B02D0022B0C
S113421810D107E0544B1A68938B43F0080323F03A
S113422810030CE0504B1A68938B23F0080343F0F7
S1134238100304E04C4B1A68938B23F01803938300
S11342480420FDF7FBFE16E09DF8082000980DF108
S1134258090100F0B5F89DF80930FE2B0BD145484B
S113426800F0C4FB9DF80A000121002200F0D4FBF1
S1134278414800F0BBFB009801A9052200F0A0F812
S113428800287FF486AE4FE0314F3B8813F4C04FCB
S113429825D013F4804F17D02E4D002128784022C2
S11342A800F0FAFA48B101AC21464022307800F017
S11342B887F80246287821462EE02878402141F2E2
S11342C8750200F061F835E001AC214630788022AF
S11342D800F076F801462046FEF744FD24E001ADDF
S11342E829468022307800F06BF804462946307855
S11342F8224600F0D1FA3B888BB92846214602228F
S1134308FFF702FC80B14FF40060FEF7B7FF022804
S11343180AD130781949172200F0BEFA04E0284679
S113432821460222FFF7F0FB074E307800F060F8D0
S11343380028A9D126B0F0BDD405002048050020E6
S1134348DC050020853D0000D9050020D8050020A3
S113435882050020A00B00201D05002078A4000081
S113436884A4000094A400004C05002090D003000D
S1134378E0050020A4A40000B4A4000028A50000BF
S113438800B502F077FC00BD10B50C4BC0B2013883
S11343981FFA81FCC0B219684FEA001E0EEB010334
S11343A81B7B81B0009092B25EF80140184611461A
S11343B802236246A04701B010BD0000E8050020B2
S11343C810B50A4BC0B20138D3F800C0C0B24FEAE6
S11343D8001E0EEB0C031B7B81B0009092B25EF8BA
S11343E80C4018460423A04701B010BDE80500207E
S11343F810B5094BC0B201381A68C0B2010101EB0B
S113440802031B7B81B000908C58184600210022BF
S11344180523A04701B010BDE805002010B50B4BDB
S1134428C0B201385FFA81FCC0B219684FEA001EB5
S11344380EEB01031B7B81B000905EF80140184627
S1134448114607236246A04701B010BDE8050020C5
S113445810B50A4BC0B20138C0B2CAB219684FEAE3
S1134468001C0CEB01031B7B81B000905CF801403D
S1134478184600210623A04701B010BDE805002016
S113448810B50B4BC0B201381FFA81FCC0B21968D1
S11344984FEA001E0EEB01031B7B81B000905EF80F
S11344A80140184611460A236246A04701B010BDD0
S11344B8E805002000B5104BC9B293F800E00F4B93
S11344C84FF0000C1B6803F1100210E052F8103C86
S11344D8834207D112F8043C8B4203D10CF1010347
S11344E8D8B207E00CF101035FFA83FC1032F445FB
S11344F8ECD1002000BD0000EC050020E8050020F8
S1134508C9B211F0100F10B59446044602D0202306
S11345180CF8013B11F0800F08D06346302203F8F1
S1134528012B78228CF8012003F1010C01F0070318
S1134538042B28BF042301F020004FEA430E0CF19A
S1134548010210E04FEA8E0334FA03F303F00F0379
S11345583033392B04D908B1073301E02733DBB2F0
S113456802F8013C01320EF1FF335FFA83FEBEF11B
S1134578FF0FE7D1501E11F0080F06D00D2302F8E3
S1134588013C0A2302F8013B104611F0400308BF1E
S113459800F8013B10BD0000013010F8013C013067
S11345A8202BFAD00138002209E0303BDBB2092B7A
S11345B802D9273B03F00F0343EA0212013010F833
S11345C8013C2F2BF1D8104670470000013000221F
S11345D805E0D30003EB42035B18A3F1300210F8A3
S11345E8011C01302F29F4D810467047C9B20023A2
S11345F801E019540133013AFBD270474FF0000C23
S113460805E01CF801300CF800300CF1010C013AFB
S1134618F7D2704700B594464FF0000E08E0734691
S11346281A5C5B5C0EF1010E9A4201D0012003E092
S1134638BCF1010CF3D2002000BD000000B501302C
S1134648013110F8012C11F8013C84469A428E4637
S113465801D001200AE09CF8003001300131002B20
S1134668EFD19EF80030181E18BF012000BD0000CD
S11346780130013111F8012C0B4600F8012C13F814
S1134688013C01300131002BF4D10138704700009E
S11346980246002000E00130835C002BFBD1704708
S11346A8F0B5044681B096B2009102F0F5FA228A78
S11346B8618A02EB06038B42C8BFC2EB0103A768F9
S11346C8C8BF9EB2E36807EB06029A42A26038BFED
S11346D8354607D3C1EB02032268A3609B1AC3EBD8
S11346E806039DB202F0E0FA39462A4603E0009830
S11346F8037801F8013C531E9AB24FF6FF73013157
S11347089A42F4D1AE420FD0C5EB060321689AB29F
S113471803E00098037801F8013C531E9AB24FF65F
S1134728FF7301319A42F4D102F0B6FA238A334472
S1134738238202F0B9FA304601B0F0BDF0B505465F
S113474881B096B2009102F0A7FA2A8A698A02EB2C
S113475806038B42C8BFC2EB0103AF68C8BF9EB251
S1134768EB6807EB06029A42AA6017D3C1EB02036F
S11347782A68AB609B1AC3EB06039CB202F094FA56
S1134788384600992246FFF739FFA6420DD0009B10
S1134798286803EB0401C4EB060204E002F084FA7F
S11347A8009938463246FFF729FF02F075FA2B8A3A
S11347B833442B8202F078FA304601B0F0BD000091
S11347C8F0B5038A92B282B0934228BF13460446D6
S11347D80F464668019343B3C26833449342436027
S11347E815D3C6EB0203019A9DB20368521B9B18AA
S11347F84360009202F058FA8FB131462A4638468F
S1134808FFF7FCFE2168009A07EB050005E002F0BB
S11348184BFA27B1019A38463146FFF7EFFE02F00A
S11348283BFA238A019A9B1A238202F03DFA0198E3
S113483802B0F0BDF0B5DCB20F4696B29DF8145044
S113484802F02AFA052C04D0062C13D0042C07D025
S11348581BE0104B1B6803EB05135B681C8A15E00F
S11348680C4B39461B68324603EB05135868FFF7AF
S1134878A7FF0EE0074B1B6803EB05135B681A6878
S11348889A605A604FF000021A82002402F00CFA6F
S11348982046F0BDE8050020F0B5C7B282B00D4649
S11348A81FFA82FE002F6AD11FFA8EFE7346CDF8D6
S11348B804E0002B3CD10A784B784C1C9A425BD11B
S11348C802F0EAF9A978394B39481970C9B2FFF7E7
S11348D8F1FDDFF8E0C08CF8000070B1364B1B68BE
S11348E803EB001353F80C0C2B79018A4A1D9B180F
S11348F8428A934204DD8CF8007002F0D5F93BE05B
S11349088B1D038221464FF0050C836811F8012C96
S11349180CF1FF3C03F8012BC2688360934224BF67
S1134928036883600131BCF1FF3FEED1062424E023
S1134938204A14785CB90A784B789A421CD18E784C
S11349481B48F1B2FFF7B6FD0446A8B104E0174BC3
S113495817701E7802F0A8F9174B29461B68019AAC
S113496803EB041353F80C0CFFF7E8FE0421044688
S113497870B201F0FFFF00E00024A0B213E0FF2FA3
S113498801D100200FE00C4B7A1E1968D2B24FEA0D
S1134998021C0CEB0103187B00925CF80140724680
S11349A829460323A04702B0F0BD0000ED0500200E
S11349B83D480000EE050020E805002000B58446C7
S11349C80CF10102C8B200E0013212F8013C002BDC
S11349D8FAD10CF10103C3EB02039AB20AB900201D
S11349E802E06146FFF758FF00BD000000B5024B26
S11349F81978FFF7E3FF00BD1D05002010B583B04B
S1134A080DF10104C9B22246FFF77AFD2046FFF7EB
S1134A18EDFF03B010BD000070B5C9B286B01646EC
S1134A280AB1944601E00DF10B0C11F0100F04D0FB
S1134A3820230CF8013B01F0FB0111EAD07204D0E9
S1134A482D23C0F100000CF8013BDFF8E8E0002555
S1134A582CE0394AAEFB02348DE818004FEAD40E34
S1134A682DB9BEF1010F0AD111F0020F01D0302384
S1134A7803E011F0040F02D020230CF8013B864513
S1134A88E7D8B0FBFEF3DBB203F130020EFB03F30D
S1134A980CF8012B284AC01AAEFB02348DE8180022
S1134AA8BEF1000F18BF01254FEAD40E0028E6D145
S1134AB8624609E02048AEFB00348DE81800302334
S1134AC84FEAD40E02F8013C2B1E18BF0123BEF195
S1134AD8000F0CBF002303F001030132002BE9D1BE
S1134AE8501E8DB911F0040F04D02023104602F88B
S1134AF8013C09E011F0020F03D0302302F8013C15
S1134B081046302300F8013B11F0080F06D0034685
S1134B180D2203F8012B0A224270581C11F040039D
S1134B2808BF037026B90DF10B00FFF75FFF0020E3
S1134B3806B070BD00CA9A3BCDCCCCCC00B50023DE
S1134B4882B08DF802308DF803308DF804008DF8AA
S1134B58051001238DF8072000200DF1020106221B
S1134B688DF80630FFF798FE02B000BD00B540B2DC
S1134B7882B0C9B288B100238DF803308DF80430AF
S1134B888DF8050001238DF8071000200DF10301AD
S1134B9805228DF80630FFF77FFE02B000BD000045
S1134BA830B58DB20446284601F054F830B100EB14
S1134BB8050320606060A060E360658230BD00008A
S1134BC8F0B5C9B282B005461046009201919FB271
S1134BD8FFF770FC30BB0021FFF76CFC0646F8B108
S1134BE8124B1B6803EB0013A3F110042B8843B189
S1134BF8384601F02FF8606018B12988FFF7D0FF14
S1134C0880B16B8843B1384601F024F8A06018B12C
S1134C186988FFF7C5FF28B1009B2360019B2373B4
S1134C28304600E0002002B0F0BD0000E805002096
S1134C3800B5C0B281B0C9B2082806D8DFE800F0D0
S1134C4816050507051E05051A00002019E0138935
S1134C586846ADF800304FF00003ADF80230136831
S1134C68094A19781423FFF7ABFF0AE0104600F04D
S1134C784DFB06E0104600F017F802E0104601F07C
S1134C88BFFC01B000BD00003D480000044BC0B2A9
S1134C9800B51870000100F0DDFF024B186000BD7C
S1134CA8EC050020E805002030B5417A04460229C5
S1134CB837D81D48FFF7FEFB002832D10021FFF743
S1134CC8F9FB054668B3201D617A174A1C23FFF7D0
S1134CD877FF30B3DFF854C06B1EDDB2DCF8003068
S1134CE828011B185A681249637A41F8232022B113
S1134CF8637A51F82320237A1376DCF800300D49BF
S1134D081B189A68637A41F8232022B1637A51F810
S1134D182320237A1376204602F0C4F96B1CD8B2F8
S1134D2800E0002030BD0000414D0000E8050020EF
S1134D38F0050020D40B0020F0B5C0B281B0DCB27D
S1134D480F46009096B29DF8185001F0A5FF042C68
S1134D580ED0052C02D0032C67D12AE0364B1B68F1
S1134D6803EB05135868838A002B5ED0058A5DE03F
S1134D78314B2A0186B91B6813449C6801F094FFDF
S1134D88032239462046FFF7D9FC054601F084FF83
S1134D98E37D13F0400F42E01B6813445868838A8C
S1134DA8002B42D0013B838239463246FFF708FD87
S1134DB83FE0002E39D0204B1B6803EB05139C6899
S1134DC8A168B7B96268914204D9638AC2EB010247
S1134DD89B1A02E003D2C1EB020398B202E0238AD1
S1134DE81BBB608AB04284BFC6EB00039DB21DD8CA
S1134DF81BE0731E01F8013BE368A160994224BFDC
S1134E082368A36001F050FF394632462046FFF775
S1134E1895FC054601F040FFE37D13F0E00F05D152
S1134E282046009902F0CEF900E0002501F03CFF8D
S1134E38284601B0F0BD0000E805002030B590F91F
S1134E482F3082B0054689B2CBB1038B8B4216D87A
S1134E5800248DF803408DF8044090F82F300DF1AC
S1134E6803018DF8053001238DF806300020223B1C
S1134E7805228DF80730FFF70FFD85F82F4002B0A3
S1134E8830BD000070B591F830300C4613F0010FB6
S1134E98C6B206D00B8B8A8C9B1A0B834FF0000387
S1134EA88B8494F82C2012F0030F16D012F0010F03
S1134EB802D03046112101E03046132103F01AFFD5
S1134EC8C0B2002840F09D8094F82C3043F0400391
S1134ED823F0030384F82C3093E012F0200F40F001
S1134EE88D80258B4DB922F04003304684F82C3050
S1134EF801F08AFF204600217DE0E3681978A36A5F
S1134F0813F4806F18D012F0040F1CBF22F00403AE
S1134F1884F82C3010D194F82E00884205D094F8E7
S1134F282D308B4208D1012D06D042F004030146EE
S1134F38012584F82C3000E0002594F8303013F073
S1134F48010F3AD0E068218B626900EB01039342B8
S1134F582ABFC0EB02030D469DB2002D51D0638BCE
S1134F68B1EB530F0BD9274BC5EB010253F826308D
S1134F785B8C9A4203DBB5EB510F88BF6D0894F83C
S1134F882C302A4643F0400384F82C30E16830463C
S1134F9801F0C8FEE36862691B189342E36028BF06
S1134FA8A368054628BFE360164B204653F826300D
S1134FB8598CFFF743FFA58423E0304603F09AFE9B
S1134FC823680133236094F82C3043F0400384F8B9
S1134FD82C30B5B9E368626901339342E36028BFB2
S1134FE8A368204628BFE360238B013B2383054B3A
S1134FF853F82630598CFFF721FF02E0304601F0C0
S113500803FF70BDF8050020034BC0B200B553F888
S11350182010FFF737FF00BD0006002010B5C0B20E
S11350280C4601F1080101F0ADFEA28C238B121A83
S11350389B1A2383E368C0EB0302A368E2609A42E5
S11350483EBF638BD318E3604FF00003A38410BD05
S113505800B50E4BC0B253F8202092F82C3039B169
S113506823F0200382F82C301146FFF70BFF0BE0E6
S113507843F0200382F82C3092F8303013F0010FFB
S113508802D01146FFF7CAFF00BD00000006002049
S1135098F0B5914BCFB253F82740904B81B053F8F9
S11350A8275094F83030C6B213F0020F1DD0628B2B
S11350B813F0080F236918BF520803EB0201A36A0F
S11350C8216113F4807F01D0531E9AB26369384674
S11350D8994222BF638BC3EB01032361216901F069
S11350E81FFEA38B0133A383ECE0A16A11F4006FC4
S11350F813D094F82C2012F0040F1CBF22F00403E0
S113510884F82C3010D194F82E30B34204BF42F006
S1135118040384F82C3000F0DC8011F0800F03D0F5
S113512894F82D30B34201D0002300E0012300930A
S1135138A36A13F0200F25D0132E12D195F830301E
S113514813F0010F03D038462946FFF767FF95F897
S11351582C3043F0200385F82C306B6801336B60E6
S1135168B7E0112E0ED195F82C3013F0200F00F073
S1135178B08023F0200385F82C3038462946FFF701
S113518881FEA6E0236801332360A36A13F4805FD9
S113519819D02A8B6B8B9A420CD82B691E702B69F9
S11351A86A69013393422B6124BFAB682B612B8B53
S11351B801332B8395F82C3013F0600F03D1384654
S11351C82946FFF75FFE009B002B45D1228B638B9A
S11351D893420ED9531C2383E38B0133E38323695E
S11351E81E702369626901339342236124BFA36853
S11351F82361A16A11F0600F26D094F82C3013F0C3
S1135208100F21D1228B238C9A421DD311F0200F29
S11352180AD095F82C30384643F0020385F82C3030
S11352282946FFF72FFE06E038464FF400714FF485
S1135238005201F009FE94F82C3043F0100384F86E
S11352482C30636801336360A26A48F2800302EA7F
S11352580303002B36D03CE0A36A13F4807F1ED0EE
S1135268E28B002A2ED0A38B0233A3832369C2EBDB
S11352780302511E626901339342236124BFA36868
S11352882361A36899423CBF638BC918E38B0B70F5
S1135298238B013323834FF00003E38312E0A38BB2
S11352A8228B0133A383638B93420BD9531C23832F
S11352B823691E702369626901339342236124BF01
S11352C8A368236194F82F0018B140B2042101F0B7
S11352D851FB01B0F0BD0000F805002000060020D5
S11352E830B585B2342000F0B5FC60B104462846D8
S11352F800F0B0FCA06030B100EB05032061E06071
S11353086361658300E00024204630BDF0B505469E
S113531881B0CEB2017A4848FFF7CCF8074618B1F5
S113532816F0040F08D183E000200021FFF7C2F82B
S1135338074608B900207CE0404B3F4A1B6816F03A
S1135348020F03EB0713A3F11000009043F8102C8D
S113535808D0E8882C7AFFF7C3FF394B009943F843
S11353682400886016F0010F12D0A888FFF7B8FF50
S11353782A7A344B43F822002B68009A13F4807F6E
S1135388506005D00369013303614FF001030383BF
S11353982B492B7A51F823203AB12B6893622B7A44
S11353A851F823206B7B82F83030DFF898E02B7AB1
S11353B85EF82320002A34D02B7B82F82F302B7AF6
S11353C8AA7B5EF823C0AB8802FB03F31E4A83FB67
S11353D802014B11ACF820302B7AEA7B5EF823C02B
S11353E8AB8802FB03F3184A83FB02014B11ACF8A8
S11353F822302B7A0C465EF823202B6893622B7A92
S11354085EF823206B7B82F830302B7A5EF82320F9
S11354186B7A82F82D302B7A5EF82320AB7A82F8E7
S11354282E3000982B7A29460373287A03F058FB08
S1135438384601B0F0BD000055540000E8050020CE
S113544800060020F80500201F85EB51F0B5DCB2FA
S113545881B0C0B2023C0F46009095B29DF8186026
S113546801F01AFC082C00F28B81DFE814F0090023
S11354789E00C50088004A018901890189011C012F
S1135488C94917F4805F14BF0B680B684FEA061408
S113549815BFE318E3189C685C68002D6DD015F0FF
S11354A8800F05D0A26A0098294601F0CDFC64E07B
S11354B815F4806F0CD0A26A2946009803F088FC82
S11354C8010A044601F001010098FFF7C1FD58E103
S11354D815F0010F19D094F8303013F0020F10D0E2
S11354E813F0080F628BA36A18BF520813F4807F65
S11354F801D0531E9AB2E2832169009801F010FC8E
S113550809E0009801F064FC05E015F0020F02D0F0
S1135518009803F039FC15F0040F03D0009803F049
S113552817FC05E015F0080F02D0009803F0FAFB09
S113553815F0100F03D0A36A43F4805305E015F067
S1135548200F03D0A36A23F48053A36215F4006FD9
S113555805D0A36A84F82D7043F4C07305E015F4EC
S1135568805F03D0A36A23F4C073A36215F0400FCD
S11355781CBF07F07F0384F82F30248D01E18A4B88
S11355881B6803EB06135868836A13F0800F08BF7F
S1135598048B00F0F680808B13F4807F08BF0446E8
S11355A800F0EF80431C5C08EBE07F4B1B6803EBC7
S11355B806139C684FB9628B238BC3EB0200A84285
S11355C8A8BF84B280F2DD80DAE001F06DFB2A46E0
S11355D8394604F10800FFF7B1F8054601F05CFB11
S11355E894F82C3013F0600F03D100982146FFF78C
S11355F849FC01F059FB54E06B4B36011B689B19BD
S11356085C6848F28013A26A02EA03033BB1A38BE5
S11356181BB901F049FB0020C3E0013BA3832A46E0
S113562804F108003946FFF7CBF894F83030054602
S113563813F0080F0CD0A38B13F0010F08D1A36843
S1135648628BE16803EB5202914238BF1346E36070
S1135658A06A10F0600F24D094F82C1011F0100FE9
S11356681FD0228B638C9A421BD821F0100310F0B0
S1135678200F84F82C300DD04B4B1B689B1999686C
S113568891F82C3043F0010381F82C300098FFF78F
S1135698F9FB06E000984FF480714FF4005201F0D2
S11356A8D3FB28467DE0012D3F494FEA061405D96E
S11356B80B6823449868AB1E9DB202E00B68234430
S11356C858687FB9012D81BF374B07601B68476055
S11356D885BF03EB06135B6840F825701F6088BF1D
S11356E85F604DE0AB0000EB0301C35C3A4602F88F
S11356F8013B4B78481C7B704378537083789370D4
S11357083EE02949340155B10B6823449B689A68E3
S11357181A61DA604FF000021A839A8330E00B684A
S11357281B195A6892F82C3013F0100F2DD023F05F
S1135738100382F82C300B681B1999688B6A13F0D4
S1135748200F09D091F82C3043F0010381F82C3054
S11357580098FFF797FB06E000984FF480714FF428
S1135768005201F071FB104B1B681B195A680CE0BE
S11357784B1C13614FF00003D3834FF001031383D1
S1135788002401F091FA20460BE04FF00003138344
S11357989383936A916813F4807F1161D160E7D190
S11357A8EEE701B0F0BD0000E8050020C0B24028D3
S11357B898BFA0F1300305D9602894BFA0F137033E
S11357C8A0F13D03D8B27047014B18607047000040
S11357D80C0600204FF4CA32002303E00133DBB285
S11357E802F580628242F9D9DBB2092B01D8303341
S11357F804E0232B01D8373300E03D33D8B2C0B2DC
S113580870470000F0B50D4F81B03B6805460BB9F1
S1135818002010E0012201AC0430002644F8043DC5
S113582801F0BAFB3E6028466946042201F0B4FB45
S113583800B10096009801B0F0BD000008060020F1
S113584810B5144B0446186881B050B106E083685B
S11358589C4202D1C06820B11AE010300368002BC2
S1135868F5D10023204669460422009302F0B6FBD2
S1135878009B13B94FF480600AE0B3F1FF3F01D1F4
S1135888002005E0044A121B9A4238BF009200988F
S113589801B010BD0C060020FBFF0300F0B581B079
S11358A806460D4600921F46FFF7CAFF044658B144
S11358B8441B09D0BC4228BF3C4606EB0500053012
S11358C80099224602F08AFB204601B0F0BD000090
S11358D870B504460D46164660B94FF4C83413E053
S11358E8002300242B601BE0201D3146012202F016
S11358F875FB15E0FFF7A4FF043020F47E7020F058
S1135908070000F580602418064B9C42E8D820461E
S1135918FFF796FF28600028E6D104F58064F3E7D2
S1135928204670BDFEFF03000A4B00B51A6842B951
S11359380AE0137900200B700BE093689842F8D0C2
S113594810321368002BF8D10430012202F046FB10
S1135958012000BD0C06002000B501F003FB00285F
S113596814BF4FF0FF30002000BD0000F0B584B034
S113597884460091174639480AB900686CE0006803
S1135988374B002832D10CF105051D6002A90DF131
S11359980F02FFF79DFF0446002850D0029B03F531
S11359A88063043323F47E7121F00701A542029138
S11359B80AD304EB01039D4206D22046FFF7CCFF2D
S11359C8029BBB423BD2ED18204602A90DF10F02FF
S11359D8FFF77EFFA8428CBF0023012300280CBFD9
S11359E8002303F0010304464BB3D7E71B6803EB1A
S11359F80002A2F5C8339B0A9BB2019302EB07038A
S1135A08A3F5C833013B9B0A9EB29B2E01D8019C87
S1135A1813E0019B9B2B1FD8C2F580279B26F6E732
S1135A28A30203F5CA352846FFF70AFF18B1011D7A
S1135A382846FFF791FF631C9CB2B442F0D1074C8F
S1135A48074B0099186823683A46C01801F0A4FA6D
S1135A58236807EB0300206004B0F0BD08060020AB
S1135A68100600200D4B30B51C68054644B90AE001
S1135A78284601F0BDF810B1A06868B903E01034F5
S1135A8821680029F4D12878FFF790FE9B2828BFC5
S1135A989B20800200F5C83030BD00000C060020B1
S1135AA8C0B2022800B504D003280DD0012815D1AE
S1135AB80BE0002002F0B8FA80B16FEA40606FEAA8
S1135AC85060C0B2002104E0002002F0ADFA28B111
S1135AD801210022002301F08FFA01E04FF0FF308A
S1135AE800BD000070B584B201200E4695B202F0E4
S1135AF89BFA38B902F098FA002808BF412080F0D0
S1135B080300C0B214F4004F1FBF6FEA40636FEA8A
S1135B185363DBB283F003006104490C32462B461D
S1135B2801F06AFA70BD000070B584B214F4004F35
S1135B380E4695B201D1012002E06404640C0020F1
S1135B4802F072FA08B9013804E0214632462B46BD
S1135B5802F04CFA70BDC0460F4B4FF000021A8099
S1135B680E4B81B019600E4B19600E4B1A7801E088
S1135B7883B1043003789342FAD1438801EB0300DC
S1135B88074B186002E0552300F8013B0DF10303AD
S1135B989842F8D901B0704714060020180600206E
S1135BA81C06002020050020054B1A68104600E05A
S1135BB801304378552BFBD0801A80B2704700001F
S1135BC81C060020034B1868034B1B68C01A80B2DC
S1135BD8704700001C06002018060020044B1868B3
S1135BE8044B1B68C01A044B1B88C01A80B2704748
S1135BF81C0600201806002014060020F0B5124EDA
S1135C08124F33683A8889B202EB03044B1E1C42D4
S1135C1818BFC1F100030E4A1CBF23405C1885B2AB
S1135C28126804EB0503934201D300200AE02046DE
S1135C3800212A46FEF7DAFC33682046C3EB040346
S1135C482B443B80F0BD00001806002014060020F9
S1135C581C060020F0B5104E104F33683A8885B200
S1135C6802EB030414F0030F0D4A1CBF24F00303D2
S1135C781C1D126804EB0503934201D300200AE0BB
S1135C88204600212A46FEF7B1FC33682046C3EBC0
S1135C9804032B443B80F0BD1806002014060020A2
S1135CA81C0600201FFA81FC48B1436993F822209E
S1135CB803EB42010132A1F81CC083F8222070478B
S1135CC8B0F81CC00246012102E0938B01315383D2
S1135CD890F8223002329942F7DB013B80F82230F7
S1135CE860467047C9B211F0010F18BF0378944693
S1135CF81CBF138002781ABF43EA02232CF8023B24
S1135D08023011F0020F1FBF0378ACF8003002789C
S1135D1843EA022314BF2CF8023B023011F0040FAB
S1135D281FBF0378ACF80030027843EA022318BF97
S1135D38ACF8003070470000044B00EBC0001B684F
S1135D4803EB800383F8211070470000200600202D
S1135D58F0B5C0B284B00190C9B20DF10E00D7B24B
S1135D681E460091FDF7E0FF01220292002590F8FB
S1135D7800E0BDF80E30CEEB0303ADF80E304378E7
S1135D88042B14D0052B25D0022B4FD1019A43792B
S1135D98934214BF00230123002A08BF43F00103E0
S1135DA81BB100230125029340E000253EE0002DAD
S1135DB83CD0009AFF2A02D08378934236D1FF2F31
S1135DC804D0C378BB4201D003252FE0002E37D07E
S1135DD802252BE0331E18BF0123002D0CBF00231E
S1135DE803F0010313B3022D14BF00240124B446A5
S1135DF815E082788B7802F07F0203F07F039A42E1
S1135E080BD19CB90B794A7943EA0222BCF80430D5
S1135E18934238BFACF8042008E00CF1080CDCF815
S1135E2800100029E5D10CB1CCF80000BDF80E3003
S1135E380BB170449BE7029B002B0CBF304600203B
S1135E4804B0F0BD30B5114B81781B6801F07F01B7
S1135E5801EBC10203EB8205EC680023FF2000225A
S1135E6801F09EFA002385F82130EB8285F8223070
S1135E781CB123822368A3606360AA682AB14FF027
S1135E880003138213689360536030BD200600201A
S1135E9830B5104A90F802C08BB212680CF07F013A
S1135EA8044601EBC10002EB8005E0782CF07F0C7E
S1135EB840EA0C00227994F805C042EA0C2201F069
S1135EC86FFAE3780BB9112300E0012385F8213038
S1135ED830BD000020060020F0B5022888B0044632
S1135EE8CDB2D7B207D11D4B294618780122002319
S1135EF8FFF72EFF2FE06846002120226E46FEF7AA
S1135F0875FB14B1012C25D110E0144B29461878DF
S1135F18FF226B46FFF71CFF002401E0FFF792FF06
S1135F2854F80D0008340028F8D113E00B4B294627
S1135F3818783A466B46FFF70BFF08B901200AE0C8
S1135F48002402E00021FFF7A3FF54F80D000834F1
S1135F580028F7D1002008B0F0BD00002406002076
S1135F6870B588B0CDB22022002106466846FEF7F7
S1135F783DFB2846FF2100226B466C46FFF7E8FEEE
S1135F8810BB012023E03EB915B9FFF75BFF1AE007
S1135F98A188FFF77DFF16E00E4B012E1A6883785F
S1135FA803F07F0303EBC30302EB830090F8213073
S1135FB80BBF43F0020303F0FD0323F0010343F096
S1135FC8010380F82130083420680028DBD108B0A8
S1135FD870BD000020060020F0B582B000931B4B72
S1135FE800EBC0001D6884002B59019197B205EBA2
S1135FF804064BB100220846394601F07BFA2B59B6
S11360083946009A98471FE0B368D3B196F8200040
S113601818B140B2042100F0ADFC96F8211011F03B
S1136028040F10D1B068438A028A9B1ABB42BCBFD2
S113603841F0040386F8213005DB01993A46FEF75E
S11360482FFB002000E0012002B0F0BD2006002054
S113605830B5426982B092F92030054689B2D3B18D
S1136068038A8B4217D800248DF803408DF8044026
S113607892F8203000208DF8053001238DF8063081
S11360880DF10301223B05228DF80730FEF704FCCD
S11360986B6983F8204002B030BD0000F0B581B0D0
S11360A800901F4688B291B203EBC302244B1B68CD
S11360B803EB8205EB8A0BB100203FE0AB8A8142F7
S11360C834BF0E4606469E428CBF6B826E82069B88
S11360D829830098698A3A46EE8201F0DFF8E86875
S11360E8698AFFF7DFFD009B6B6022E0EB6823B150
S11360F85B6993F82230012B1FD83846069901F0C2
S113610809F9D0B9C4EB06039EB2009B3A461B19A1
S1136118AC8A1846B44228BF344621460093069BED
S113612801F0BCF82146E868FFF7BCFD6B8AE41867
S11361386C826C8AEB8AA342D8D1E88A01B0F0BD9C
S113614820060020F0B5C0B289B00D4602921F4661
S1136158062800F24582DFE810F0C0001C02150290
S11361680700230231023702029A02EBC203DFF866
S11361787824126802EB8305E98AEC68002900F0A8
S11361882F826B8A8B42C0F08480002C64D0268ACC
S1136198002E61D06069FFF793FDC0EB06006269C9
S11361A880B2208292F822104B001A33D2180023AE
S11361B800E053880139023AB1F1FF3FF9D19EB2A8
S11361C8B04227D1002E41D1EB8AA98AB3FBF1F260
S11361D801FB02F29B1A9BB22BB900200021029A00
S11361E83B4601F05BF86368EA8A1A44E368626034
S11361F89A4224BF638AC3EB0203626928BF6360BF
S11362084FF00003EB8292F8213023F0400382F828
S113621821301BE06368EA8A1A44E36862609A42A0
S113622822BF638AC3EB020363606068E3684FF0CC
S113623800021B1A99B2238AEA829B1B8B42B8BFBD
S113624899B20A46029B0097FFF728FF6369204624
S1136258198AFFF7FDFEC3E1AA8AB1FBF2F302FB38
S113626803F3C3EB01039BB27BB92B8B8B4206D19F
S1136278029B53B195F8213013F0100F05D100207B
S11362880021029A3B4601F009F84FF00001E98227
S1136298A6E1C3EB0103AA8A9BB2934234BF1E460C
S11362A8164654B16069FFF70BFD238A1B1A238233
S11362B863692046198AFFF7CBFE6B68688A314602
S11362C8C018029A3B4600F0E9FF20463146FFF722
S11362D8E9FC6B8A33446B8282E12B78C24A0393CC
S11362E8166803994FF00003F38221F08003012B11
S11362F800F0B880032B00F00281002B40F03181BC
S11363082B781C46092B00F29E80DFE803F0999C49
S11363189C9C9C66059C96692A782B7842EA032CF7
S11363282B7818462B782A7819462B7842EA0322C8
S11363380CF47F43B3F5007F049210D003DCB3F56B
S1136348807F23D106E0B3F5407F0DD0B3F5C06F4D
S11363581CD116E00DF12200FDF7DEFC0DE00DF175
S11363682200FDF7E1FC08E05FFA8CF00DF1220150
S1136378FDF7E2FC002800F02F81BDF822100097F9
S113638802E09A4800970A21049ADAE03368002B5D
S113639800F0228140EA0124062202212846CDF891
S11363A804C001F0A7F80399034603F8011BDDF8BC
S11363B804C0591C4FEA1C2280F801C05A70481CBA
S11363C84C70240A4470049B421C5370049902388C
S11363D80B0A9370844B1B68CFE02B78BB74FDE0E9
S11363E829780020FFF7BCFD0446002840F0F4801B
S11363F87F4B2A781A707C4B1B6893F82060002E18
S113640800F0EC802946012207A8FEF7F7F8752367
S11364188DF8193002238DF81A300020043B0DF151
S1136428160107228DF816408DF817408DF818606C
S11364388DF81B30FEF730FAD0E06D4800974BE03A
S11364486C4800977BE03368002B00F0C58002227B
S11364582846062101F04EF8039A634B02704470F3
S11364681B688AE02B781C46002B38D00A2B1DD0D9
S11364780B2B39D15E4B1B78002B00F0AD802846DE
S113648803210DF11E02FFF72DFC9DF82010FF22B9
S11364980020FFF721FD9DF820109DF81E20012003
S11364A8FFF71AFD002840F0978097E0504B1B78BF
S11364B8002B00F09180284602210DF12202FFF7FB
S11364C811FC9DF8221002200022FFF705FD002888
S11364D800F08280033000970121012231E0444B0F
S11364E81B78002B78D028E03368002B74D028461A
S11364F80621022200F0FEFF039B03702FE02B7895
S11365081C4613BB284602210DF12202FFF7EAFBC1
S1136518374B1B781BB9BDF82230002B5CD1BDF872
S1136528223003EBC30306EB830393F8213013F003
S1136538080F02D03048009701E030480097022144
S113654802220023FFF7AAFD4AE03368002B43D058
S113655802222846062100F0CDFF039A02704470F7
S113656809E03368002B37D001222846072100F0C0
S1136578C1FF039A02701C490B68398A1B68002200
S113658898472EE01B8A23B9029829460022022341
S113659803E03A8A029829460123FFF71DFD20E00B
S11365A89B7C33B1104BCF211B6893F92000FEF775
S11365B8DDFA00200021FFF7D3FC11E00A4BCE21BD
S11365C81B6893F9200004E0074BCD211B6893F95D
S11365D82000FEF7CBFA03E0042002E0032000E0E9
S11365E8002009B0F0BD00002006002074A50000BA
S11365F8240600202606002072A5000070A50000CD
S1136608F0B50446264E18230430A17B254A356884
S1136618FEF7D6FAA37B074633B103EBC30305EBB6
S11366288300A389838211E00020214601F062FBE4
S1136638607C00EBC00080002430FFF70BFB4FF0B8
S1136648080330608382A37C80F82030164B4FEA1D
S1136658071C1B68634453F8083CC36013B15861B2
S113666823890382A37B8376A37B53B1E17B41B166
S11366780B4A01EBC103126802EB83008176A389FC
S11366888382094B1B68634453F80C3C83601BB139
S11366985861A37C80F82030236803603846F0BD35
S11366A820060020B5660000E8050020F0B5DCB23D
S11366B887B0C0B2023C0E46019097B29DF83050A4
S11366C800F0EAFA042C00F2B180DFE804F00328B1
S11366D87B219F00584B16F4805F14BF1B681B680E
S11366E84FEA051215BFD318D3189A685A6817F0D9
S11366F8400F09D0516991F8213013F0010F1CBFE4
S113670806F07F0381F82030536993F821608EE006
S1136718494B1B6803EB05135B681E8A87E0464BED
S11367281B6803EB05139D6865B902AC0198214603
S113673800F0F0FD002879D100F0B6FA3046394669
S113674800943AE06B6993F8213013F0010F6DD08F
S113675846B96A8A2B8AC3EB0200B842A8BF86B23C
S113676865DA63E000F0A0FA31463A462846FDF7B8
S1136778E5FF064600F090FA6B6993F8213013F0B0
S1136788400F54D102AF0198394600F0C3FD0028E8
S11367984DD16B68EC686A69E41A92F82130A4B2A6
S11367A843F04003A64238BF344682F82130A4B2ED
S11367B800F07AFA6868214600970A46019BFFF7B9
S11367C86DFC37E01C4B31461B683A4603EB051356
S11367D85C682046FDF7F4FF6369054693F82130A9
S11367E813F0040F10D000F057FA626992F82130C0
S11367F823F0040382F821306369987E00F04CFD8D
S11368080028F9D000F050FA284613E00A4B2A0170
S11368181FB11B6813449A6802E01B6813445A6842
S11368281368936053604FF000031382002600F04E
S11368383BFA304607B0F0BDE8050020054B1B883D
S113684803F00100C0F1000000F4344080EA530072
S11368587047000038060020144B154A196813685D
S11368680133136001B31AE011F8033CBBB1104BB8
S11368781A6851F8083C9A4211D1C37B022B04D000
S11368880423C37311F8043C037482892AB151F8B0
S1136898083C9B1841F8083C01E001F8032C0C3132
S11368A851F80C0C0028DFD1704700003006002096
S11368B8DC0B0020104B30B51C6840B2DCB10F4B28
S11368C81D6815E01B78834211D10CE09D4209D163
S11368D800F0E2F90023237263720223EB7300F0E1
S11368E8E3F908E00C342368002BEFD103E01435F6
S11368F82B68002BE6D130BD30060020340600207A
S1136908194BF0B51D6840B28EB2D7B2002D29D00C
S1136918164B1C6823E01B7883421FD11AE09C4263
S113692817D100F0B9F9E37B23F00203E3732F7264
S11369381FB9A68126B96E7208E0002E08BF012689
S11369480B4B1B689B196B6001236B7200F0ACF94D
S113695808E00C352B68002BE1D103E014342368DC
S1136968002BD8D1F0BD00003006002034060020EA
S1136978DC0B0020134B30B51D68134B40B21C6868
S1136988C9B21AE01B78834216D199B97DB911E0CE
S11369989C420BD100F080F90C4BA2891B689B1810
S11369A86B600023E37300F07FF909E00C352B6872
S11369B8002BEDD1E17303E014342368002BE1D1FB
S11369C830BD00003006002034060020DC0B002017
S11369D830B51C4B82B01D682DE0EB7B13F0050F1E
S11369E828D000F059F9AB891BB9EB7B13F0010FE0
S11369F81BD12B7CA3B100248DF803408DF80440EF
S1136A082B6800201B788DF806408DF805302B7C08
S1136A180DF1030105228DF80730FDF73DFF2C74B5
S1136A28EB7B13F0020308BFEB7300F03DF96B68CE
S1136A382846984714352B68002BCED1024B18688A
S1136A4802B030BD3406002028060020F0B5D2B2CA
S1136A5884B0614B009200221A60604B01901A6066
S1136A685F4B1A7858E05BB2934250D10A4600E073
S1136A782246144614F9013F002BF9D1C1EB020355
S1136A88DFB207EB870080000430FFF7E3F8534BCD
S1136A98E41B0026054684464FF0000E1860029455
S1136AA803962BE0019924E0227843B29A421FD13D
S1136AB84B68CCF80040CCF804300B89ACF80830AB
S1136AC81BB1039A531CDBB203934B89ACF80A300D
S1136AD88A89ACF80C208B7B8CF80F30BCF80A3010
S1136AE80BB993B20BB1731CDEB20CF1140C03E0B6
S1136AF810310C68002CD7D10EF1010E029B1EF840
S1136B0803000028CED1CCF8000055B956E011F89E
S1136B18013F002BFBD101310B78002BA3D10027B7
S1136B284CE0002E2ED006EB46008000043080B2E4
S1136B38FFF790F8284B1860284B1A6819E0518918
S1136B4849B14FF6FF73994204BF00235381538917
S1136B580121436005E0938913B10121436002E0F8
S1136B68002143680BB10123437209B140F80C2B8F
S1136B7814321368002BE2D106EB4603164AA0EB45
S1136B8883031360039A009B02EB0300C0B2FEF771
S1136B987DF8039A92B1114B1C680CE023894BB120
S1136BA8032001212246FEF743F8A07310B94FF0E1
S1136BB8FF33A37314342368002BEFD1094801F081
S1136BC8B1FA094B00241C6000F078F8074B3846EA
S1136BD81C6004B0F0BD000030060020340600201C
S1136BE82005002038060020DC0B002028060020A1
S1136BF800B5002286460EE012F80EC09C4509D066
S1136C08602B01D9203B02E0402B09D92033DBB2A9
S1136C189C4505D10132535C90B2002BECD100E0C5
S1136C28002000BD0F4B43F820200F4A00F11F033A
S1136C3800EA020213EA200338BF0346002AC9B255
S1136C484FEA631C05DA013A6FEAC2626FEAD2625C
S1136C58013201239340054A42F82C30044BC154B5
S1136C6870470000400200201F00008000E100E09F
S1136C7800E400E0074B00221A6002F1804202F5AA
S1136C88BA2202F57E720432136883F0010313609A
S1136C98704700000C00004072B6024A13680133C2
S1136CA8136070477C070020034A1368013B136094
S1136CB803B962B6704700007C070020094A0A4BF2
S1136CC81A6003F18043094AA3F55E43143BDA636F
S1136CD8074A136843F0E0631360064B07221A60FF
S1136CE8704700009F25260014E000E04D83000053
S1136CF820ED00E010E000E0C0B200B510B10128BA
S1136D0809D103E0044A0520062102E0034A0620CB
S1136D180621FFF787FF00BDE9800000A580000079
S1136D287047000092B2C0B2FAB110B101281CD168
S1136D3803E00F484FF4007C02E00E484FF4000CC7
S1136D48B2F5806F28BF4FF48062013A92B201EB2A
S1136D5802030360084B110141EA03038360013213
S1136D68064B90B2C3F800C000E000207047000052
S1136D789000002070010020018000C028F00F401E
S1136D8800207047C0B210B101281DD108E00F4B94
S1136D984FF400721A6002F10052A2F5B87207E0CB
S1136DA80A4B4FF400021A6002F1FC5202F5B87261
S1136DB8936813F0070F07D0926843F6F07302EA5A
S1136DC803031B09581C00E0002070472CF00F40F7
S1136DD8C0B2C2B210B52AB1094B012A0CBF1C4675
S1136DE8002400E0074CFFF787FF10236364A36BBC
S1136DF843F01003A363236B43F40073236310BDB0
S1136E0800D0004000C0004070470000C0B210B17C
S1136E18012816D10AE021B10A4A136823F00203B3
S1136E280EE0084A136843F0020309E021B1054A59
S1136E38136823F0010303E0024A136843F00103D3
S1136E4813607047FCB3054030B58DB215F4C05FCC
S1136E58C4B25ED015F4006F2DD014B1012C26D124
S1136E6813E0354A136843F008031360A2F522229D
S1136E78A2F53E620C3A136843F002031360A2F5CC
S1136E888E72136843F0020310E02B4A136843F030
S1136E9808031360A2F52222A2F53E620C3A136895
S1136EA823431360A2F58E721368234313602046AC
S1136EB80021FFF7ABFF15F4805F2AD014B1012C31
S1136EC827D113E01C4A136843F001031360A2F5A9
S1136ED82422A2F5DF520C3A136843F00803136026
S1136EE8A2F58E72136823F0080311E0124A13689E
S1136EF823431360A2F52422A2F5DF520C3A136847
S1136F0843F080031360A2F58E72136823F08003A4
S1136F18136040F2011305EA030313B1204601216B
S1136F2806E040F2022305EA03031BB120460021D0
S1136F38FFF76CFF30BD000008E10F40074B1A60F3
S1136F48043B1960064A40F0244343F48403136065
S1136F58034B1B680342FBD17047000004D00F4069
S1136F6808D00F4030B520F47E740D4624F0070491
S1136F78084B002202201A602146FFF7DFFFB5F50F
S1136F88806F04D904F58064A5F58065F0E70020D6
S1136F9830BD00000C00004070B520F003042368E5
S1136FA81546001B4E1C17E0C100FF228A4023EA45
S1136FB8020216F8013C8B40032842EA030309D174
S1136FC8012021461A46FFF7B9FF65B154F8043F7A
S1136FD8002000E001300136013DE5D201202146C0
S1136FE81A46FFF7ABFF002070BD000000B54FF450
S1136FF80061FFF7B7FF00BDF0B5C0B282B09EB222
S1137008552310F0800F00928FB28DF8073001D10C
S1137018002502E000F07F00012510F0400F0AD09F
S11370284FF4C030FFF7E2FF4FF4C430FFF7DEFF40
S11370384FF4C03405E0022814BF4FF4C0344FF4B1
S1137048C4347EB94DB1B4F5C03F14BF4FF4C03059
S11370584FF4C430FFF7CAFF19E02046FFF7C6FF14
S1137068AFB11BE004EB0700009932460230FFF78A
S113707893FF20460DF107010122FFF78DFF6DB93B
S1137088601C0DF107010122FFF786FF06E0204688
S11370980DF107010122FFF77FFFF1E7002002B09D
S11370A8F0BD000030B5417A0546CAB22AB13E4B5C
S11370B8012A0CBF1C46002400E03C4C002931D1B5
S11370C83B4A08201368042143F002031360C03AC2
S11370D8136823F002031360136823F00203136098
S11370E8BC32136843F480531360C03A136823F422
S11370F880531360A2F52422A2F54262043A13686D
S113710843F00C031360FC32136843F00C03136060
S1137118103A136843F00C031360264B01221A60DB
S1137128254A30E0224A25201368042143F001034C
S11371381360C03A136823F001031360136823F043
S113714801031360BC32136843F480431360C03AEC
S1137158136823F480431360A2F52422A2F5E152B4
S1137168043A136843F0C0031360FC32136843F015
S1137178C0031360103A136843F0C00313600F4B45
S113718801221A600E4AFFF74DFD28881023322881
S1137198236206D0B0F5C87F01D1052302E0182385
S11371A800E03123E36030BD0010024000000240DB
S11371B808E10F401C000240C17F00001C1002407F
S11371C89D7F0000C9B2CAB232B1304B012A0CBF4C
S11371D89C464FF0000C01E0DFF8B4C0436813F894
S11371E8012B8275C2684360934224BF03684360DD
S11371F8436813F8012BCCF80020C268436093421B
S113720824BF03684360DCF8003013F0010F1BD07F
S1137218837D012B01D1072300E00B23CCF8043034
S11372286FF03F03C375038A4268033B0382194B1B
S113723853F8211012F8013B0B76C36842609A4256
S113724824BF0368436020E0436813F8012BCCF89B
S113725808204360837D012B01D1072300E0032329
S1137268CCF804300123CCF810304268C3689A4241
S113727828BF0368827D28BF43604023C375038AFF
S11372889B1A013B013A0382827570470010024041
S113729800000240F00500200120704710B589B2B3
S11372A804469E4610466AB9184A137813F0010F2B
S11372B808D04023137005E0DEF80C2014F8013BD5
S11372C8137000E08C460CF1FF331FFA83FC4FF671
S11372D8FF739C45F0D198B908290D490AD103F1E7
S11372E8804303F5802303F58073022203331A7065
S11372F8CA7409E0054A0A2313700423CB7403E013
S1137308DEF804200123137010BD000002010540BB
S1137318800B002003280AD8DFE800F0020B1621AE
S1137328164B1B7813F0020F26D1154BCB600020A7
S113733823E0144A137813F0010F1DD1124BCB60CC
S1137348124B1B68043314E0114A137813F0010F2D
S113735812D1104BCB600D4B1B68083309E00E4A61
S1137368137813F0010F07D10C4BCB60074B1B6844
S11373780C338B604A60DAE702207047020105404B
S1137388200005401201054024000540980B002008
S11373982201054028000540320105402C00054023
S11373A8484BF0B55FFA81FCD3F800E0012303FAF7
S11373B80CF3C0B2FF2894B2DDB20ED1424B43495C
S11373C804221A700B886FEA050292B213400B80EC
S11373D802310B8813400B8073E03B4B05221A7073
S11373E8033383F800C00CF1FF334FEA8C01DBB29E
S11373F80EEB01062EF801404FEAC30C2246082181
S113740803E053009AB24B1ED9B2B2F5006FF8D319
S113741820F08003012B4FEA5C0703D00CDB032B1D
S11374280ADC02E04FF0400E08E010F0800F18BFAD
S11374384FF0000E05D11DE04FF0000E10F0800F44
S11374481AD0234B234A197013882B431380224ADA
S11374581388224ADB081380214B002223F81740A3
S113746807330CF803204EF02002043B0CF80320E9
S1137478164A1BE04FF0100E1A4B1B4A197013885A
S11374882B431380144A1388184ADB081380184BBB
S1137498002223F81740013B0CF8032002F1804234
S11374A8043302F5A0220CF803E0083213880A49D1
S11374B82B4313800B8832889B180B800023F370AE
S11374C8B370F0BD980B00200B0005400600054082
S11374D862000540420305409C0B002064000540FF
S11374E8100105406300054040030540660005405F
S11374F814010540844689B292B204E09CF8003035
S11375088354531C9AB24B1E99B24FF6FF73994297
S11375180148F3D170470000800700201E4A012368
S113752830B513601D4B00201A6805E022B11C4BCE
S113753801301B6822F8023B1A4B1B6813F4807F46
S1137548F4D0DFF864C0DFF854E0BCF80010CEF8DB
S113755800200129154D0CD8154A164C136823F43C
S113756880331360012323602B689847002323602A
S113757811E02B681BB14B1EACF8003003E0A2EB02
S11375884003CEF800300C4B1B6813F00F0F02D1E8
S11375980A4B01221A6030BD0C8003407807002092
S11375A8488003404C800340740700207007002083
S11375B800E10F407C07002014800340288003402A
S11375C8F0B5037985B0012B064600F0FE8003D39D
S11375D8022B40F0A0824AE1C27901239340DDB234
S11375E8002D00F098828379072B08D8DFE803F090
S11375F8090C0F1215181B04DFF8204515E00024A8
S113760813E0DFF81C4510E0DFF818450DE0DFF85B
S113761818450AE0DFF8144507E0DFF8144504E0EC
S1137628DFF8104501E0DFF81045082B00F27382FB
S1137638DFE803F0050E172029323B444D00DFF83C
S1137648FC34DFF8FCC403EB82070020012147E087
S1137658DFF8F034DFF8F0C403EB820701200221DD
S11376683EE0DFF8E834DFF8E8C403EB82070220E1
S1137678042135E0DFF8DC34DFF8DCC403EB8207EF
S1137688032008212CE0DFF8D434DFF8D4C403EB5A
S113769882070420102123E0DFF8C834DFF8C8C4C7
S11376A803EB82071E2020211AE0DFF8C034DFF83C
S11376B8C0C403EB82071F20402111E0DFF8B43473
S11376C8DFF8B4C403EB82072020802108E0DFF848
S11376D8AC34DFF8ACC403EB820736204FF4807176
S11376E833688BB9737A082B0ED0636923EA0503D0
S11376F86361002B40F00F8203F1604303F560439C
S1137708022203F5C07302E2DFF8782413680B43FE
S11377181360C03A136823EA01031360636A6FEACB
S113772805010B4063626368A2680B406360D4F888
S113773820312B43C4F82031337A012B10D902EAC3
S11377480103A360337A042BE36802D12B43E3607B
S113775815E00B40E360337A2269032B09D00BE070
S1137768E3680B40E36042EA0503A360337A2269C5
S113777813B942EA050301E002EA01032361737ABB
S1137788022B09D0082B0CD0012B13D1D4F81431B7
S11377982B43C4F814310DE0D4F818312B43C4F842
S11377A81831F94B1B6813F0020F0AD1F74B10225A
S11377B81A6006E0256271796246FFF733FA336886
S11377C83B6063692B436361A5E1847A032C00F36E
S11377D8A2814FF4803202FA04FCED4902F180429E
S11377E80B6802F56E2243EA0C030B6002F5827201
S11377F8230303F180451368022C43EA0C0305F5BF
S11378084035136001DD232002E0630003F1130017
S1137818DF4A136823EA0C031360336853B1DD4B62
S1137828717953F82420FFF7FDF9DB4B326843F8EC
S113783824200123AB61F38813F0020F01D0022343
S113784800E001236B60F388328913F0010F14BF41
S11378584CF25033322302FB03F3AB62F38813F088
S1137868080F01D0212300E00123EB6053E10369F1
S113787813F4801F15D0C94B00221A6003F50C338A
S113788803F5A4631A6003F580531A6002F1804279
S113789802F57E2202F58072136823F480331360A4
S11378A839E113F4804F0FD0816969B1828A06E007
S11378B8BB4B1B681AB121F8023B531E9AB2B94B51
S11378C81B6813F4807FF3D0316911F4805C40F0B5
S11378D8228111F4004F00F01481B34AB3481368AD
S11378E843F480331360F268B3680092B04A01939A
S11378F8136823F001031360036823F00F02AD4BF0
S1137908026001EA0303002B69D011F4403F2BD035
S113791833698DF80CC003F44033B3F5003FCDF858
S113792808C007D0B3F5403F06D0B3F5803F06D171
S1137938032302E0022300E004238DF8103001231E
S11379488DF80E3002238DF80D3004238DF80F3096
S113795802A808238DF81130FFF732FE934A136802
S113796843F0040313603BE011F0404313D0B3F138
S1137978004F09D0B3F1404F0AD0B3F1804F08BF8C
S113798842F0010302D02BE042F00203036027E037
S113799842F00303FAE711F0005F18BF42F0050351
S11379A8F4D111F048631BD0B3F1806F0ED003D823
S11379B8B3F5000F14D106E0B3F1006F09D0B3F1A9
S11379C8406F0DD108E042F00603DFE742F00703F9
S11379D8DCE742F00803D9E742F00903D6E702607E
S11379E8B27D754B00241A604FF0000E00254FF04D
S11379F8000C0122019800994FEA420740EA01036A
S1137A081A4231D00A420CD01CF0010F0FD1A30046
S1137A1801229A4015434FEA5C029A404EEA020E4C
S1137A2804E0A3000CFA03F34EEA030E0134BCF19C
S1137A38030F0CD9534ACCF10B0113685F4843F088
S1137A480803136001238B4002681A431CE04D4A63
S1137A58CCF1070113685A4843F01003136001235B
S1137A688B4002681A431EE0BCF1030F0ED9454B44
S1137A781B6813F0080F18D0CCF10B0101238B40BD
S1137A884E48026822EA030202600EE03D4B1B687E
S1137A9813F0100F3DD0CCF1070101238B40484867
S1137AA8026822EA0302026033E0BCF1070F3A4697
S1137AB802D00CF1010C9DE7002C2CD0631E9B0016
S1137AC806229A403F4B45EA0202C3F800E0043319
S1137AD81A6071793C4A0E20FFF7A4F832683B4BD0
S1137AE81A603B4BB28A1A80B2693A4B1A602B4A25
S1137AF8136843F001031360083A136843F0010361
S1137B081360336913F0100F05D0334B01221A6048
S1137B1801E03A46CDE705B0F0BD0000FCF30540AE
S1137B28FC830540FC930540FCA30540FCB30540D9
S1137B38FCC30540FCD30540FCE305404006002097
S1137B48898600006006002039860000800600202F
S1137B58ED850000A0060020A1850000C0060020D5
S1137B6855850000E0060020098500000007002074
S1137B78BD84000020070020718400004007002015
S1137B882584000008E10F4000E100E01C94054052
S1137B9844E00F40E4A5000060070020088003408B
S1137BA8488003404C80034000E10F4014800340A8
S1137BB800800340000083EC3080034028B5054072
S1137BC828C5054040800340257500007007002043
S1137BD87407002078070020288003400C4A1368A3
S1137BE843F00803136002F15A4202F53D02094BBF
S1137BF802F58A6201321A6000224FF080431A604B
S1137C0802F1804208320223136003231360FEE763
S1137C1800E10F40000C004070470000704700006E
S1137C28704700007047000070470000704700006C
S1137C3870470000704700007047000081B000EBF7
S1137C4880000090009B013B0093009BB3F1FF3F31
S1137C58F8D101B070470000164A174B1749C2EB18
S1137C68030003E011F8013C02F8013C144B013213
S1137C78034401319A42F5D1124A134B1349C2EB1A
S1137C88030003E011F8013C02F8013C104B0132F7
S1137C98034401319A42F5D10E4A0F4BC2EB03015A
S1137CA802E0002302F8013C0C4B01320B449A42D7
S1137CB8F7D170471C0500204805002044A60000A1
S1137CC81D05002008200000BC8E000008200000CC
S1137CD80920000048050020C80F0020490500209D
S1137CE84FF0000E2EE27047D0F800D0D0F804F020
S1137CF870470000454810B503680C4643F48033C8
S1137D08434903600B68434A23F480330B601368C8
S1137D1881B023F4804313600368A2F51E2243F064
S1137D28800303600B68A2F5446223F080030B60B0
S1137D38103A136843F018031360FC32136843F0D5
S1137D48180313600C3A136843F010031360637C40
S1137D580133DBB2042B637401D904236374607C9C
S1137D688000FDF777FF2C4B4FF0080218602B4B6F
S1137D7802804FF001021A8004331B78284A0093CA
S1137D88284B2C201B8804219BB20093264B1B886C
S1137D989BB20093FEF746FF244B04221A70244B2F
S1137DA81B6813F0800FFAD0638913F0020F18D1FF
S1137DB8204A136843F004031360043A136843F039
S1137DC80403136002F59072136843F0040313600C
S1137DD8194B01221A60A3F5826340220B3B1A70E7
S1137DE812E0144A136843F004031360043A136856
S1137DF823F00403136002F59072136843F004033C
S1137E0813600D4B00221A6001B010BD08E10F4049
S1137E1848E00F4070E00F40980B00200600054032
S1137E28D586000002000540040005400B0005400B
S1137E3850E00F4000F405401C04054030B5D2B2B0
S1137E4805460C4672B6194910460B682A46013392
S1137E580B60E1682346FEF775F90138052820D838
S1137E68DFE800F0121F03161F0D002000212A4628
S1137E782346FFF713FAA5B92023E37411E00C4B4A
S1137E8840221A70E2740CE0FEF70EFF01200BE0AA
S1137E98074A202313701023E37428460821FDF7AA
S1137EA84BFFFEF701FF002030BD00007C070020D7
S1137EB802010540F0B592F917300E46002B14461E
S1137EC8C7B2957D35DA314ADDB16B1EA37552F818
S1137ED82710B2688B6803F8012B8B60A37D0BB95C
S1137EE8052300E009237360284B53F82700038A0D
S1137EF8826801330382C3689A4224BF036883609B
S1137F0842E052F82720938A107E0133938250B1BD
S1137F1872B61F4B40B21A68042101321A60FEF788
S1137F2829FDFEF7C1FE238A002B29D13561E575A9
S1137F382AE09DB16B1E9375536813F8012B8A6070
S1137F486360A37D0BB9052300E0012362687360B5
S1137F58E3689A4224BF2368636015E0138A7BB9F7
S1137F680B61107ED37578B172B6094B40B21A68AA
S1137F78042101321A60FEF7FDFCFEF795FE03E0CA
S1137F8820463946FFF71EF9F0BD0000F005002031
S1137F987C070020054B01221A60054B00B55A687E
S1137FA801200449FFF786FF00BD00001C100240B1
S1137FB8D40B002000100240054B01221A60054B27
S1137FC800B51A6800200449FFF774FF00BD0000DB
S1137FD81C000240D40B002000000240034600B5F8
S1137FE808461946FCF70AFB00BD000070B5C0B28C
S1137FF889B2022814BF4FF4C0304FF4C43040187B
S11380089EB2851C07E0541C284611460122FFF73E
S1138018E5FF01352246731E9EB24FF6FF739E425A
S1138028F1D1002070BD000010B581B0C4B20222A5
S11380384FF4C0300DF10201FFF7D0FF9DF8023074
S1138048002C0CBFFF245524552B05D19DF8033073
S1138058A34201D1012011E002224FF4C4300DF1F2
S11380680201FFF7BBFF9DF80230552B05D19DF89F
S11380780330A34201D1022000E0002001B010BD6A
S1138088054B01211B6800B581EAD31101F00101F8
S11380980120FCF7DDFF00BDFC83054010B516E0A8
S11380A8236813F0100F08D00B4B10221A60443BBE
S11380B818680121C0B2FCF7EBFF236813F0200F06
S11380C805D0054B20221A600120FCF79DFF034CC4
S11380D82368002BE4D110BD44D0004040D00040B8
S11380E810B516E0236813F0100F08D00B4B1022BC
S11380F81A60443B18680021C0B2FCF7C9FF236822
S113810813F0200F05D0054B20221A600020FCF73D
S11381187BFF034C2368002BE4D110BD44C000400E
S113812840C00040064B10B51C682388038013B96F
S113813841F27B230380FEF781FB208010BD000001
S1138148940B002010B5664B81B00DF102021A6041
S1138158644A136823F480031360136843F40063C8
S11381681360136823F0F06323F47C7313601368BB
S113817843F0C07343F460731360136823F400532B
S11381881360136843F480031360574B1B6813F0A0
S1138198400FFAD0534A136823F40063136002F1C2
S11381A85F4202F57002514B02F5065220321A6002
S11381B84F4BD3604F4B13614F4B53614F4B9361FC
S11381C84F4B13634F4B93604F4B93634F4BD362A7
S11381D840324F4B13604F4B9A4201D00432F8E7B8
S11381E84D4C4FF400532360FFF736FD4B4B4FF0D3
S11381F8FF321A6003F57863012218331A604FF0CE
S1138208005204331A60236802F1005243F0200339
S113821802F57E22236048321368414923F0200383
S11382281360B832136843F008031360C03A136844
S113823823F0080313603B4B4FF480720B6003F187
S1138248145303F54C1303F5F65307331A6002F17C
S11382580E7202F5862202F558724FF080431A60B6
S113826802F17852A2F57012A2F55052583A02233C
S113827813600323136003F18043002209331A6057
S11382880A60F9F7D1FE284B31221A60274B1C6883
S11382986CB927482749FDF75FFC274827490A2274
S11382A8FEF7D4FBFEF794FB04460028FAD02268B4
S11382B80AB9204905E0224B18689047014600286E
S11382C8E7D06068FDF748FCA068E1680A22FEF779
S11382D8BDFBFEF77DFB04460028FAD0E7E7000063
S11382E8940B002060E00F4050E00F4008ED00E0E0
S11382F8217C0000257C0000297C00002D7C0000E6
S1138308317C0000357C0000397C00003D7C000095
S1138318417C0000EC02002008E10F406CE00F40B3
S1138328000C004051E5CC1A40E10F40280600201B
S113833880A50000C80F002094A5000088A50000AF
S11383482C060020074B4FF0007200B51A6072B675
S1138358054A136801331360FEF77EFAFEF7A4FC9E
S113836800BD000004ED00E07C070020074B01225B
S113837800B51A6072B6064A136801331360054BD8
S1138388DB689847FEF790FC00BD000024300340EA
S11383987C07002060070020074B012200B51A6003
S11383A872B6064A136801331360054B9B689847F5
S11383B8FEF77AFC00BD0000242003407C0700205F
S11383C860070020074B012200B51A6072B6064AFE
S11383D8136801331360054B5B689847FEF764FC28
S11383E800BD0000241003407C0700206007002023
S11383F8074B012200B51A6072B6064A13680133A6
S11384081360054B1B689847FEF74EFC00BD00003F
S1138418240003407C0700206007002030B50D4C81
S1138428802512E013681D420AD00B4B1D6072B6FA
S11384380A4A136801331360E3699847FEF734FC6A
S1138448074B043C6D089C4203D0064A1368002B72
S1138458E8D130BD400700201C0406407C070020FA
S1138468200700201804064030B50D4C802512E082
S113847813681D420AD00B4B1D6072B60A4A136872
S113848801331360E3699847FEF70EFC074B043C7D
S11384986D089C4203D0064A1368002BE8D130BD0E
S11384A8200700201CF405407C070020000700205A
S11384B818F4054030B50D4C802512E013681D42B0
S11384C80AD00B4B1D6072B60A4A13680133136055
S11384D8E3699847FEF7E8FB074B043C6D089C42A8
S11384E803D0064A1368002BE8D130BD00070020EA
S11384F81CE405407C070020E006002018E4054041
S113850830B50D4C802512E013681D420AD00B4B80
S11385181D6072B60A4A136801331360E369984709
S1138528FEF7C2FB074B043C6D089C4203D0064A85
S11385381368002BE8D130BDE00600201CD40540A8
S11385487C070020C006002018D4054030B50D4C27
S1138558802512E013681D420AD00B4B1D6072B6C9
S11385680A4A136801331360E3699847FEF79CFBD2
S1138578074B043C6D089C4203D0064A1368002B41
S1138588E8D130BDC00600201CC405407C0700208B
S1138598A006002018C4054030B50D4C802512E013
S11385A813681D420AD00B4B1D6072B60A4A136841
S11385B801331360E3699847FEF776FB074B043CE5
S11385C86D089C4203D0064A1368002BE8D130BDDD
S11385D8A00600201CB405407C070020800600206B
S11385E818B4054030B50D4C802512E013681D42BF
S11385F80AD00B4B1D6072B60A4A13680133136024
S1138608E3699847FEF750FB074B043C6D089C420E
S113861803D0064A1368002BE8D130BD8006002039
S11386281CA405407C0700206006002018A405400F
S113863830B50E4C802513E013681D420BD00C4B4B
S1138648E1691D6039B172B60A4A136801331360CF
S11386588847FEF729FB084B043C6D089C4203D06D
S1138668064A1368002BE7D130BD000060060020DD
S11386781C9405407C0700204006002018940540FF
S113868830B50D4C802512E013681D420AD00B4BFF
S11386981D6072B60A4A136801331360E369984788
S11386A8FEF702FB074B043C6D089C4203D0064AC4
S11386B81368002BE8D130BD400600201C84054017
S11386C87C0700202006002018840540F0B5F048F7
S11386D881B003684921EF4AD15401330360EE4B5A
S11386E8EE4F1A783B781A40009259D0E84DE94980
S11386F82B684822CA54009A013396B216F0040F24
S11387082B601CD0E64B4FF04001198004233B70CA
S113871872B6E44AE44C1368002101331360042060
S113872800222346FDF70EFDFEF7BEFA0023A374CC
S1138738E374D8492B685222CA5401332B6016F0CB
S1138748010F14D006233B7072B6D64A0021136871
S113875805200133136000220023FDF7F3FCFEF724
S1138768A3FA2B68CB495322CA5401332B6016F061
S1138778020FB4D005233B7072B6CA4A00211368AD
S113878806200133136000220023FDF7DBFCFEF70B
S11387988BFA2B68BF497222CA5401332B609EE7B7
S11387A8C24B1B889EB2C24B1B8816EA030700F013
S11387B8158116F0010F00F0D580B54CDFF8D4C24E
S11387C8236830220CF803200133320A0CF8032002
S11387D8DFF8E0E201330CF803609EF8002001336F
S11387E80CF80320B04A0133D07C591C10F0060F52
S11387F80CF8030021600FD09EF8003013F0100F1E
S11388080AD06FF07F038EF80030009BD37458238E
S11388180CF801304B1CDFE0042873D006D801287B
S11388285DD011D3022840F09D803DE0102800F06F
S1138838968003D8082840F095806BE0202800F043
S11388488480402840F08E809A4D2B7813F0010FD5
S113885800F088808F4C4323635403F18043DFF88E
S113886830E203F5A0234A1CC433CEF800200133B8
S11388781B788D4902F1010C0B8283B13033A35468
S11388888D4B4028CB608D4BCEF800C01B684D60E3
S11388988B6034D000200022FFF7D0FA62E0302346
S11388A8A354CEF800C05DE07A4B41225A54784B69
S11388B84A1C1A607C4B804ADA60E2325A607F4A6A
S11388C812689A6072B6774903200A6801320A600E
S11388D800210022FDF736FCFEF7E6F942E06D4878
S11388E85223435403F1804303F5A023B6331B7882
S11388F84A1C6D4983540B82654B01321A6000206F
S11389080222C9E7634B54225A54614B4A1C1A6029
S1138918082225E05F485323435403F180434A1C4B
S113892803F5A0235A49B4330A6001331B785E4D1A
S11389381C462B82B3B98354531C0B600020294670
S11389480222FFF77BFAEC740CE0524B61225A5472
S11389584F4B4A1C1A60544B9A7C594B1A7000228C
S1138968514BDA7416F00E0F3FF4B9AE484C494D2A
S113897822687423AB54013216F0020F226003D02C
S11389883123AB54531C236016F0040F1CD0236806
S113899832224C49EA540A780133EA5401332360F9
S11389A8494A414BDA60454A5960126808329A606C
S11389B872B63C4903200A6801320A600021022287
S11389C8FDF7C0FBFEF770F916F0080F3FF487AE09
S11389D823683322EA540133236080E63B4B2C4856
S11389E81B88DFF8B0C09CB2394B1B881C423FD0AF
S11389F8026872230CF80230013214F0020F02608C
S1138A0824D03123334D0CF802302B7801320CF882
S1138A180230013202602B7813F0010F16D022497C
S1138A282D4B4D60CB60254B1B6804338B602B4B5F
S1138A381B889BB20CF802300B82531C0360012282
S1138A480120FFF7FBF9012818BF2F7014F0040F59
S1138A5806D00F480F4A03683221D154013303600A
S1138A6814F0080F3FF43BAE09483321036832E69B
S1138A78036820220CF8032002F5647201330632DD
S1138A889342036002DD024B00221A6001B0F0BD7C
S1138A983C060020E00B00200A0005400B000540BE
S1138AA89C0B00207C070020800B0020020005405E
S1138AB8060005400201054020000540980B0020EF
S1138AC80000054022010540280005400400054037
S1138AD8080005401601054024000540180105401A
S1138AE8C0B2C2B230B50D462AB17D4B012A0CBFC3
S1138AF81C46002400E07B4C0023236318B10128A2
S1138B0840F08C8044E0784A136843F00103136012
S1138B18C03A136823F001031360136823F00103B8
S1138B281360BC32136843F001031360C03A13683E
S1138B3823F001031360A2F52422A2F5E152043ABA
S1138B48136843F003031360FC32136843F0030310
S1138B5813606B7B13F0010F60D0A2F59822634B6E
S1138B68A2F5A2620C3A5A6003F1005303F57E237E
S1138B7803F57A634FF4007204331A60183B1A60E1
S1138B8808331A60A3F572230222A3F57C6343E039
S1138B98554A136843F004031360C03A136823F07A
S1138BA804031360136823F004031360BC321368CE
S1138BB843F002031360C03A136823F002031360FE
S1138BC8A2F52222A2F5E152043A136843F0C00345
S1138BD81360FC32136843F0C00313606B7B13F01B
S1138BE8010F1BD0A2F59A22414BA2F5A2620C3ABE
S1138BF85A6003F1005303F57E2303F56C634FF4C5
S1138C08000204331A60183B1A6008331A60A3F58B
S1138C1870230222A3F5FE531C3B1A602B6813F041
S1138C28400F04D04FF4C0510022FEF70DF9EB7A3F
S1138C380B2B28D8DFE803F00C1014181C20242769
S1138C482A2D06091B22082325E00D22242322E0CD
S1138C5842F6B0022B231EE041F2584215231AE0D3
S1138C6840F62C220B2316E040F21652052312E09C
S1138C7840F28B2203230EE040F2451221230AE03E
S1138C88D922012307E0A222312304E05122182328
S1138C9801E0362210236262A3622B6813F00602F5
S1138CA808BFE26206D013F0040F01D0022300E0EB
S1138CB80623E3622B6813F0100F1EBFE36A43F028
S1138CC80803E3622B6813F0010FE36A14BF43F04F
S1138CD8400343F06003E3620123236330BD0000D3
S1138CE800D0004000C0004008E10F409000002080
S1138CF870010020C0B2C9B228B1084B01280CBFCA
S1138D081846002000E00648836913F0800F01D15B
S1138D18012001E0016000207047000000D00040FD
S1138D2800C00040C0B228B1074B01280CBF184648
S1138D38002000E00548836B23F020038363036B62
S1138D4823F480730363704700D0004000C00040E0
S1138D58C0B2C2B210B52AB1094B012A0CBF1C46D5
S1138D68002400E0074CFDF7C7FF20236364A36BCE
S1138D7843F02003A363236B43F48073236310BD80
S1138D8800D0004000C00040C0B228B1074B012801
S1138D980CBF1846002000E00548836B23F010033D
S1138DA88363036B23F400730363704700D00040AC
S1138DB800C00040054B01211B6800B581EAD301BE
S1138DC801F001010020FCF743F900BDFC830540D4
S1138DD810B589B211F00C0F83B0C4B225D011F0CC
S1138DE804031CBF264B53F8243000220093254B60
S1138DF81B5D8DF80630244B13F804E0234B185DF3
S1138E08D1B24B1C013250FA03FCF9D101238DF87D
S1138E180930684604238DF807108DF808308DF85A
S1138E2805E08DF804C0FEF7CBFB194B1A68154B07
S1138E38195D01238B401A4215D0072913D8DFE89E
S1138E4801F00406080A0C0E1014124B0EE0124B23
S1138E580CE0124B0AE0124B08E0124B06E0124BEE
S1138E6804E0124B02E0002008E0114B074A1B689B
S1138E78125D134208BF4FF48070F4D103B010BDE3
S1138E88F4A50000FCA50000FEA5000000A6000053
S1138E9808E10F40FC830540FC930540FCA3054012
S1138EA8FCB30540FCC30540FCD30540FCE3054086
S1078EB8FCF305407E
S1138EBC56312E332E303131000000000D0A0A4891
S1138ECC656C6C6F2C20776F726C642E2E2E204C7C
S1138EDC4D335333373438204556414C0D0A00007A
S1138EEC4144432056616C7565733A0D0A000000C9
S1138EFC3D3D3D3D3D3D3D3D3D3D3D000D0A5361F8
S1138F0C6D706C652D00000066617669636F6E2E62
S1138F1C69636F0008007800202017005D0A0000C8
S1138F2C000041444D494E002020755461736B651B
S1138F3C7226755461736B6572204E756D62657221
S1138F4C2031000000000050140103000000000058
S1138F5C148F000007000000C38F00007E04000083
S1138F6C00000000000000000000000000000000F1
S1138F7C1800000000000000C0A80003FFFFFF0061
S1138F8CC0A80001C0A80001436F6D6D616E642020
S1138F9C6C696E6520626C6F636B65640D0A00000E
S1138FAC436F6E6E656374696F6E2074696D65646E
S1138FBC206F75740D0A00000001000100101000F0
S1138FCC00010020006804000016000000280000C6
S1138FDC0010000000200000000100200000000030
S1138FEC0000000000130B0000130B000000000035
S1138FFC0000000000FFFFFFFFFFFFFFFFFFFFFF6C
S113900CFFFFFFFFFFFFFFFFFFFFFFFFFFFFFFFF60
S113901CFFFFFFFFFFFFFFFFFFFFFFFFFFFFFFFF50
S113902CFFFFFFFFFFFFFFFFFFFFFFFFFFFFFFFF40
S113903CFFFFFFFFFFFFFFFFFFFFFFFFFFFFFFFF30
S113904CFFFFFFFFFFD7DBDDFF919CA2FF5F6F7774
S113905CFF5F6F77FF5F6F77FF5F6F77FF5F6F77F0
S113906CFF5F6F77FF5F6F77FF5F6F77FF919CA256
S113907CFFFFFFFFFFFFFFFFFFFFFFFFFFFFFFFFF0
S113908CFFA5AEB3FF5F6F77FF5F6F77FF5F6F77FF
S113909CFF5F6F77FF5F6F77FF5F6F77FF5F6F77B0
S11390ACFF5F6F77FF5F6F77FF5F6F77FF5F6F77A0
S11390BCFFFFFFFFFFFFFFFFFFFFFFFFFFA5AEB3A7
S11390CCFF5F6F77FF5F6F77FF879399FFD7DBDDC8
S11390DCFFFFFFFFFFFFFFFFFFFFFFFFFFFFFFFF90
S11390ECFFFFFFFFFFFFFFFFFF5F6F77FF5F6F77F0
S11390FCFFFFFFFFFFFFFFFFFFD7DBDDFF5F6F7796
S113910CFF5F6F77FFAFB7BBFFFFFFFFFFFFFFFFF3
S113911CFFFFFFFFFFEBEDEEFFAFB7BBFFC3C9CC07
S113912CFFFFFFFFFFFFFFFFFF5F6F77FF5F6F77AF
S113913CFFFFFFFFFFFFFFFFFF919CA2FF5F6F7715
S113914CFF879399FFFFFFFFFFE1E4E5FF919CA2EA
S113915CFFFFFFFFFFD7DBDDFF5F6F77FF8793997F
S113916CFFFFFFFFFFFFFFFFFF5F6F77FF5F6F776F
S113917CFFFFFFFFFFFFFFFFFF5F6F77FF5F6F775F
S113918CFFD7DBDDFFFFFFFFFF7D8A91FF879399FC
S113919CFFFFFFFFFFD7DBDDFF5F6F77FF8793993F
S11391ACFFFFFFFFFFFFFFFFFF5F6F77FF5F6F772F
S11391BCFFFFFFFFFFFFFFFFFF5F6F77FF5F6F771F
S11391CCFFFFFFFFFFE1E4E5FF5F6F77FF879399F4
S11391DCFFFFFFFFFFD7DBDDFF5F6F77FF879399FF
S11391ECFFFFFFFFFFFFFFFFFF5F6F77FF5F6F77EF
S11391FCFFFFFFFFFFFFFFFFFF5F6F77FF5F6F77DF
S113920CFFFFFFFFFFD7DBDDFF5F6F77FF879399CE
S113921CFFFFFFFFFFD7DBDDFF5F6F77FF879399BE
S113922CFFFFFFFFFFFFFFFFFF5F6F77FF5F6F77AE
S113923CFFFFFFFFFFFFFFFFFF5F6F77FF5F6F779E
S113924CFFFFFFFFFFD7DBDDFF5F6F77FF8793998E
S113925CFFFFFFFFFFD7DBDDFF5F6F77FF8793997E
S113926CFFFFFFFFFFCDD2D4FF5F6F77FF5F6F77F8
S113927CFFFFFFFFFFFFFFFFFF5F6F77FF5F6F775E
S113928CFFFFFFFFFFD7DBDDFF5F6F77FF8793994E
S113929CFFFFFFFFFFD7DBDDFF5F6F77FF8793993E
S11392ACFFFFFFFFFF879399FF5F6F77FF919CA2EE
S11392BCFFFFFFFFFFFFFFFFFF5F6F77FF5F6F771E
S11392CCFFFFFFFFFFD7DBDDFF5F6F77FF8793990E
S11392DCFFFFFFFFFFD7DBDDFF5F6F77FF879399FE
S11392ECFF9BA5AAFF5F6F77FF5F6F77FFD7DBDD6F
S11392FCFFFFFFFFFFFFFFFFFF5F6F77FF5F6F77DE
S113930CFFFFFFFFFFD7DBDDFF5F6F77FF879399CD
S113931CFFFFFFFFFFD7DBDDFF5F6F77FF879399BD
S113932CFF5F6F77FF5F6F77FFAFB7BBFFFFFFFF89
S113933CFFFFFFFFFFFFFFFFFF5F6F77FF5F6F779D
S113934CFFFFFFFFFFD7DBDDFF5F6F77FF5F6F77FB
S113935CFF5F6F77FF5F6F77FF5F6F77FF5F6F77ED
S113936CFF5F6F77FFAFB7BBFFFFFFFFFFFFFFFF91
S113937CFFFFFFFFFFFFFFFFFF5F6F77FF5F6F775D
S113938CFFFFFFFFFFD7DBDDFF919CA2FF5F6F7731
S113939CFF5F6F77FF5F6F77FF697880FF9BA5AAEC
S11393ACFFE1E4E5FFFFFFFFFFFFFFFFFFFFFFFF10
S11393BCFFFFFFFFFFFFFFFFFFFFFFFFFFFFFFFFAD
S11393CCFFFFFFFFFFFFFFFFFFFFFFFFFFFFFFFF9D
S11393DCFFFFFFFFFFFFFFFFFFFFFFFFFFFFFFFF8D
S11393ECFFFFFFFFFFFFFFFFFFFFFFFFFFFFFFFF7D
S11393FCFFFFFFFFFF000000000000000000000062
S113940C000000000000000000000000000000004C
S113941C000000000000000000000000000000003C
S113942C000000000000000000000000000000002C
S113943C0000000000000000202D2000656E616219
S113944C6C65640D0A00000064697361626C656488
S113945C0D0A00000D0A42414420464F524D41541E
S113946C202D207175697474696E670D0A000000F3
S113947C0D0A424144204C454E475448202D20713E
S113948C75697474696E670D0A0000003000000081
S113949C446F776E6C6F6164696E672E2E000000EA
S11394AC2A0000000D0A5465726D696E617465645E
S11394BC2C20726573657474696E672E2E2E0000F1
S11394CC0A0D53657269616C206E756D6265723A32
S11394DC20000000536F66747761726520766572A4
S11394EC73696F6E200000004465766963652069BA
S11394FC64656E74696669636174696F6E3A2000A1
S113950C0A0A0D000A0D3D3D3D3D3D3D3D3D3D3DB1
S113951C3D3D3D3D3D3D3D3D3D0A0D00656E616269
S113952C6C65000064697361626C65000D0A496EB8
S113953C76616C6964207377697463680D0A000042
S113954C0A0D53797374656D206D656D6F72792096
S113955C7573653A0A0D00003D3D3D3D3D3D3D3D75
S113956C3D3D3D3D3D3D3D3D3D3D0A0D0000000072
S113957C467265652068656170203D20000000001E
S113958C2066726F6D2000000A0D556E757365644C
S113959C20737461636B203D200000000D0A546835
S11395AC652064657669636520686173206265650E
S11395BC6E206F7065726174696E6720666F7220BD
S11395CC0000000042616420706F7274206E756D2F
S11395DC6265720D0A0000000D0A506F72742064EB
S11395EC6972656374696F6E3A2000004F5554506C
S11395FC55540D0A00000000494E5055540D0A00F4
S113960C496E76616C696420706F72740D0A000087
S113961C506F727420697320696E7075740D0A0032
S113962C506F72742073746174653A2000000000EA
S113963C310D0A00300D0A000D0A3F3F0D0A2300BC
S113964C436F6E6E656374696E6720555342207761
S113965C697468205253323332202D206469736349
S113966C6F6E6E6563742055534220746F20717550
S113967C69742E2E2E0D0A00506C6561736520756D
S113968C73652055534220636F6E6E656374696F06
S113969C6E21210D0A000000506C65617365207306
S11396AC7461727420646F776E6C6F61643A00003D
S11396BC0A0D427965204279650A0D000A0D506144
S11396CC72616D65746572207365740A0D00000017
S11396DC0A0D54656D702E20506172616D65746550
S11396EC72207365740A0D000A0D506172616D6508
S11396FC7465722076616C7565203D200000000055
S113970C0A0D4E6F2076616C696420706172616D14
S113971C657465727320617661696C61626C650A4B
S113972C0D0000000A0D4F726967696E616C207040
S113973C6172616D657465727320726573746F7296
S113974C65640A0D000000000A0D466163746F72B3
S113975C7920706172616D657465727320726573C2
S113976C746F7265640A0D000A0D506172616D6547
S113977C7465727320696E76616C69646174656476
S113978C0A0D00000A0D4E657720506172616D65FB
S113979C746572732076616C6964617465640A0D16
S11397AC000000000A0D436F6E6669677572617480
S11397BC696F6E2073617665640A0D00496E636F80
S11397CC72726563742064617461206C656E677475
S11397DC680D0A000D0A53657269616C20636F6E23
S11397EC66696775726174696F6E0D0A000000001A
S11397FC42617564203D2000696E76616C69642158
S113980C000000003700000038000000204269749A
S113981C730D0A00207061726974790D0A000000DE
S113982C2073746F70206269742873290D0A000008
S113983C466C6F7720636F6E74726F6C200000003F
S113984C486967682077617465722000250D0A00E9
S113985C4C6F772077617465722000000D0A536594
S113986C6375726974792073657474696E67730DAA
S113987C0A0000005465726D696E616C206D656E32
S113988C75206C6F67696E00465450207365727650
S113989C657200005745422073657276657200004C
S11398AC57454220736572766572206175746865DC
S11398BC6E7469636174696F6E00000054454C4E9C
S11398CC4554207365727665720000002020205484
S11398DC656C6E657420706F7274206E756D626544
S11398EC72203D2000000000496E636F7272656344
S11398FC742073657269616C2073706565640D0AFC
S113990C00000000496E636F7272656374207061AD
S113991C726974790D0A0000496E636F7272656323
S113992C742073746F7020626974730D0A000000E4
S113993C496E636F727265637420666C6F77206313
S113994C6F6E74726F6C0D0A000000000A0D4152A8
S113995C50207265736F6C7665640A0D000000000C
S113996C0A0D415250207265736F6C7574696F6E79
S113997C206661696C65640A0D00000020202020BB
S113998C204D61696E206D656E750000204C414E52
S113999C20636F6E66696775726174696F6E00001F
S11399AC20202053657269616C20636F6E66696751
S11399BC2E00000020496E7075742F4F75747075ED
S11399CC74206D656E75000020202041646D696EF5
S11399DC2E206D656E750000202020537461747305
S11399EC2E206D656E7500002020202055534220DA
S11399FC6D656E75000000004D41430031000000A0
S1139A0C436F6E666967757265204C414E20696EB2
S1139A1C746572666163650032000000436F6E66A4
S1139A2C69677572652073657269616C20696E74FF
S1139A3C657266616365000033000000476F207433
S1139A4C6F20492F4F206D656E75000034000000A7
S1139A5C476F20746F2061646D696E6973747261F1
S1139A6C74696F6E206D656E750000003500000022
S1139A7C476F20746F206F766572766965772F73E4
S1139A8C746174697374696373206D656E75000019
S1139A9C36000000476F20746F20555342206D65CB
S1139AAC6E75000068656C7000000000446973708A
S1139ABC6C6179206D656E75207370656369666978
S1139ACC632068656C700000717569740000000097
S1139ADC4C6561766520636F6D6D616E64206D6F8E
S1139AEC6465000075700000676F20746F206D61F1
S1139AFC696E206D656E75007365745F6468637060
S1139B0C000000003C656E61626C652F64697361D2
S1139B1C626C653E20444843500000007365745FDA
S1139B2C69705F616464000053657420495020615E
S1139B3C64647265737300007365745F69705F6D40
S1139B4C61736B00536574204950207375626E65A4
S1139B5C74206D61736B00007365745F69705F676B
S1139B6C776179005365742064656661756C742043
S1139B7C67617465776179007365745F6574685F98
S1139B8C7370656564000000536574204C414E206D
S1139B9C7370656564202831302F3130302F415576
S1139BAC544F290073686F775F636F6E6669670043
S1139BBC53686F77206E6574776F726B20636F6E6A
S1139BCC66696775726174696F6E000073686F778C
S1139BDC5F636F6E6669675F6F00000053686F7731
S1139BEC206F726967696E616C206E6574776F7231
S1139BFC6B20636F6E66696775726174696F6E0052
S1139C0C73617665000000005361766520636F6EA6
S1139C1C66696775726174696F6E20746F20464C47
S1139C2C4153480076616C696461746500000000FE
S1139C3C56616C69646174652074656D706F7261D2
S1139C4C727920636F6E6669672E20696E20464CAC
S1139C5C41534800617270202D610000526571758A
S1139C6C65737420415250207461626C650000006D
S1139C7C617270202D64000044656C65746520412C
S1139C8C5250207461626C65000000007365745F4F
S1139C9C6261756400000000536574207365726919
S1139CAC616C20626175642072617465000000004F
S1139CBC7365745F73746F700000000053657420D7
S1139CCC73746F7020626974732028312F312E35B0
S1139CDC2F3229007365745F62697473000000008D
S1139CEC536574206461746120626974732028372D
S1139CFC2F3829007365745F70617200536574208A
S1139D0C70617269747920284556454E2F4F44442E
S1139D1C2F4E4F4E452900007365745F666C6F7748
S1139D2C0000000053657420666C6F7720636F6EBF
S1139D3C74726F6C2028584F4E2F5254532F4E4F21
S1139D4C4E4529007365745F686967685F77617451
S1139D5C6572000053657420666C6F7720737461B0
S1139D6C6C6C20282529205B312E2E39395D00009E
S1139D7C7365745F6C6F775F776174657200000054
S1139D8C53657420666C6F7720726573746172749A
S1139D9C20282529205B312E2E39395D0000000046
S1139DAC53686F772073657269616C20636F6E669C
S1139DBC696775726174696F6E0000007365745F16
S1139DCC6464720053657420706F727420747970BB
S1139DDC65205B312E2E345D205B3C693E7C3C6FF0
S1139DEC3E0000006765745F64647200476574200C
S1139DFC6461746120646972656374696F6E205B5D
S1139E0C312E2E345D000000726561645F706F72D8
S1139E1C740000005265616420706F727420696E66
S1139E2C707574205B312E2E345D0000777269746A
S1139E3C655F706F7274000053657420706F727478
S1139E4C206F7574707574205B312E2E345D205B1D
S1139E5C302F315D000000005361766520706F7205
S1139E6C742073657474696E67206173206465660D
S1139E7C61756C74000000007365745F6674700027
S1139E8C3C656E61626C652F64697361626C653EDE
S1139E9C2046545020736572766572007365745F46
S1139EAC74656C6E657400003C656E61626C652F44
S1139EBC64697361626C653E2054656C6E657420D4
S1139ECC73657276696365007365745F77656200A8
S1139EDC3C656E61626C652F64697361626C653E8E
S1139EEC2057454220736572766572007365745F02
S1139EFC7765625F61757468000000003C656E6193
S1139F0C626C652F64697361626C653E20574542CF
S1139F1C207365727665722061757468656E7469F8
S1139F2C636174696F6E000053686F7720636F6EA2
S1139F3C66696775726174696F6E000072656A6533
S1139F4C637400005265736574206E6F6E2D7361BB
S1139F5C766564206368616E6765730072657374FB
S1139F6C6F726500526573746F72652066616374F9
S1139F7C6F72792073657474696E677300000000E6
S1139F8C72657365740000005265736574206465B2
S1139F9C7669636500000000697073746174000075
S1139FAC53686F772045746865726E65742073749A
S1139FBC617469737469637300000000725F697083
S1139FCC73746174000000005265736574204574E9
S1139FDC6865726E657420737461746973746963F3
S1139FEC7300000075705F74696D650053686F775A
S1139FFC206F7065726174696E672074696D650099
S113A00C6D656D6F7279000053686F77206D656DA7
S113A01C6F727920757365007573622D736572693F
S113A02C616C000052533233323C2D3E5553422066
S113A03C6D6F64652028646973636F6E6E656374F9
S113A04C20746F2071756974290000007573622D7A
S113A05C6C6F6164000000005553422D535720640B
S113A06C6F776E6C6F6164000820080060A10000BB
S113A07C0F08000088990000C0A10000140E000015
S113A08C9899000068A20000160C0000AC9900001E
S113A09CF8A200000F080000C099000058A30000AB
S113A0AC110C0000D4990000E8A300001107000073
S113A0BCE49900003CA400000D050000F499000094
S113A0CC049A000000000000040900003330300042
S113A0DC0000003630300000000031323030000017
S113A0EC0032343030000000343830300000003995
S113A0FC3630300000003134343030000031393225
S113A10C30300000333834303000003537363030DE
S113A11C00003131353230300032333034303000DD
S113A12C4F444400004556454E004E4F4E450031B9
S113A13C000000312E3500320000004E4F4E450019
S113A14C0000005254530000000000584F4E000011
S113A15C00000000089A00000C9A000000040000A3
S113A16C249A0000289A000000050000449A00007C
S113A17C489A000000060000589A00005C9A0000FF
S113A18C00070000789A00007C9A00000009000087
S113A19C9C9A0000A09A0000000A0000B09A0000EB
S113A1ACB89A000000000000D49A0000DC9A000069
S113A1BC02000000F09A0000F49A0000000D000068
S113A1CC049B0000109B000007010000289B00006A
S113A1DC349B000004010000449B0000509B0000D1
S113A1EC04020000649B0000709B00000403000048
S113A1FC849B0000949B000004060000B09B0000AC
S113A20CBC9B000004050000D89B0000E89B0000E8
S113A21C040A00000C9C0000149C000003060000BF
S113A22C309C00003C9C000003050000609C000076
S113A23C689C0000040700007C9C0000849C0000C7
S113A24C04080000B09A0000B89A00000000000056
S113A25CD49A0000DC9A000002000000F09A00007E
S113A26CF49A0000000D0000989C0000A49C0000CF
S113A27C05000000BC9C0000C89C00000501000007
S113A28CE09C0000EC9C000005020000009D000016
S113A29C089D000005030000249D0000309D000073
S113A2AC05040000509D0000609D00000515000091
S113A2BC7C9D00008C9D000005160000B09B0000E6
S113A2CCAC9D0000051100000C9C0000149C0000C7
S113A2DC03060000B09A0000B89A000000000000C9
S113A2ECD49A0000DC9A000002000000F09A0000EE
S113A2FCF49A0000000D0000C89D0000D09D0000E1
S113A30C01020000F09D0000F89D0000010B00000C
S113A31C149E0000209E000001040000389E0000E2
S113A32C449E0000010500000C9C0000649E00008B
S113A33C010C0000B09A0000B89A00000000000064
S113A34CD49A0000DC9A000002000000F09A00008D
S113A35CF49A0000000D0000849E00008C9E000006
S113A36C07020000A89E0000B49E00000700000035
S113A37CD49E0000DC9E000007030000F89E000041
S113A38C089F000007050000B09B0000349F0000EC
S113A39C060200000C9C0000149C00000306000044
S113A3AC489F0000509F000003070000689F0000B6
S113A3BC709F0000030200008C9F0000949F00001B
S113A3CC01000000B09A0000B89A000000000000E0
S113A3DCD49A0000DC9A000002000000F09A0000FD
S113A3ECF49A0000000D0000A49F0000AC9F000034
S113A3FC04040000C89F0000D49F0000040B00005C
S113A40CF09F0000F89F0000010A00000CA000005F
S113A41C14A0000001010000B09A0000B89A0000DA
S113A42C00000000D49A0000DC9A00000200000036
S113A43CF09A0000F49A0000000D000024A0000023
S113A44C30A000000800000058A0000064A0000028
S113A45C08010000B09A0000B89A00000000000047
S113A46CD49A0000DC9A00000200000055534220EC
S113A47C52657365740A0D005553422053757370FD
S113A48C656E6465640A0D005553422052657375FC
S113A49C6D650A0D00000000456E756D6572617482
S113A4AC6564202800000000290A0D003FA5000067
S113A4BC43A500004DA500005DA500005EA50000AD
S113A4CC68A5000009024300020104C0000904004D
S113A4DC00010202000505240010010524010100FD
S113A4EC0424020205240600010705830340000A24
S113A4FC09040100020A00000507050102400000DE
S113A50C070582024000001201100102000008BE7F
S113A51C1C0101000101020301000000436F6D6D79
S113A52C616E64206C696E6520626C6F636B65642C
S113A53C0D0A00040309040A034D0061006E007542
S113A54C0010034D0079002000500072006F00646D
S113A55C00000A0343006F006E0066000803490004
S113A56C6E007400000001000A06000200000040A6
S113A57C01000000010058660000000001577561DD
S113A58C6D4E73000000000004A600008943000017
S113A59C00000000040001000CA600005123000080
S113A5AC450002000000000010A600007D3C0000E5
S113A5BC2500FFFF000000001CA60000913E0000D7
S113A5CC2500FFFF00000000000000000000000058
S113A5DC0000000000000000F9830000CD8300009F
S113A5ECA183000075830000BD8D000089800000EC
S113A5FC000003030880000057646F67000000002C
S113A60C617070006D61696E74656E6163650000E4
S113A61C7573620048544D004A5047004749460040
S113A62C435353004A53000042494E0054585400BB
S10BA63C49434F003F3F3F007A
S113A644FFFF00000100000020A6000024A6000073
S113A65428A600002CA6000030A6000034A60000A2
S10FA66438A600003CA6000040A6000040
S903814D2E
